:020000040000FA
:040200006BEF03F0AD
:040208000EEF01F004
:080218002DEF01F0D8CF01F039
:10022000E0CF02F0006EF3CF03F0F4CF04F0F0ACB7
:100230001DEF01F0F0B0C9EC0BF0A2A023EF01F02C
:10024000A1B071EC09F003C0F3FF04C0F4FF00504B
:1002500002C0E0FF01C0D8FF1000D8CF06F0E8CF01
:1002600005F0E0CF07F0F3CF08F0F4CF09F0F0BCD1
:100270003DEF01F0F0B0C9EC0BF0A2B043EF01F09C
:10028000A1B071EC09F0A2B04CEF01F0AECFE8FFE5
:100290006ECFE8FF52EF01F09EBAC8EC0FF0A4BA9F
:1002A00033EC10F008C0F3FF09C0F4FF07C0E0FF13
:0A02B00005C0E8FF06C0D8FF1000EB
:10030000F95000011150F926DAEF2BF0DCEF2BF059
:10031000E9EF2BF0FEEF2BF00CEF2CF01AEF2CF0A6
:1003200028EF2CF036EF2CF046EF2CF054EF2CF0A9
:1003300062EF2CF064EF2CF012000009D8A4A7EFB4
:1003400001F00001000E0F6E000E106E1200E806A4
:10035000030B0A0DF9CFE8FFF350F92685C00FF023
:1003600086C010F0120087C00FF088C010F0120095
:1003700089C00FF08AC010F012008BC00FF08CC043
:0403800010F0120067
:10040000EFCFE8FFE806070B0A0DF9CFE8FFF3503E
:10041000F9263EC050F03FC051F012003CC050F0F1
:100420003DC051F0120040C050F041C051F01200E8
:1004300042C050F043C051F0120044C050F045C0DB
:1004400051F0120046C050F047C051F0120048C0B1
:1004500050F049C051F012004AC050F04BC051F06A
:1004600012000F0B060DF9CFE8FFF350F926BBC2BF
:10047000E8FF1200BCC2E8FF1200BDC2E8FF120094
:10048000BEC2E8FF1200BFC2E8FF1200C0C2E8FF10
:100490001200C1C2E8FF1200C2C2E8FF1200C3C2CC
:1004A000E8FF1200C4C2E8FF1200C5C2E8FF120054
:1004B000C6C2E8FF1200C7C2E8FF1200C8C2E8FFC8
:0E04C0001200C9C2E8FF1200CAC2E8FF120013
:100500000001E806070B0A0DF9CFE8FFF350F926C2
:1005100099510D6E9A510E6E12009B510D6E9C51A9
:100520000E6E12009D510D6E9E510E6E12009F5167
:100530000D6EA0510E6E1200A1510D6EA2510E6EE5
:100540001200A3510D6EA4510E6E1200A5510D6E36
:10055000A6510E6E1200A7510D6EA8510E6E12001C
:100600000001E8BE33EF03F0E806070B0A0DF9CF4F
:10061000E8FFF350F9260D5075270E50762312008F
:100620000D5077270E50782312000D5079270E5069
:100630007A2312000D507B270E507C2312000D50A0
:100640007D270E507E2312000D507F270E508023F1
:1006500012000D5081270E50822312000D50832767
:100660000E5084231200E806070B0A0DF9CFE8FFAD
:10067000F350F9260D50756F0E50766F12000D5025
:10068000776F0E50786F12000D50796F0E507A6FA1
:1006900012000D507B6F0E507C6F12000D507D6F5D
:1006A0000E507E6F12000D507F6F0E50806F120043
:1006B0000D50816F0E50826F12000D50836F0E50DF
:1006C000846F1200F2AE12000001010EAD6FAD6733
:1006D00067EF03F012000BEC0CF0928802C5E8FF04
:1006E000E81EE86676EF03F092988098939C819CD0
:1006F00000015D6A5E6A0001566A640E00EC0CF04F
:10070000280EE8CFD4F20001500E386EC30E396EB9
:100710000F018350306E316E326E0F018450336E94
:10072000346E356E0F0199908780949693948296DB
:1007300081940001000E176E000E186E0001000E6D
:10074000196E000E1A6E0001000E1B6E000E1C6E5C
:100750000001000E1D6E000E1E6E0001000E136ED5
:10076000000E146E0001000E156E000E166E0001D4
:10077000000EB76F000EB86F0001000EB96F000ECB
:10078000BA6F0001000EBB6F000EBC6F0001000EBF
:10079000BD6F000EBE6F0001606B616B626BAD6B75
:1007A000AE6BAF6BF369F56B0201BA6B0101116BB4
:1007B0000001D86B16EC35F0020100510001B16F59
:1007C000040EEBEC08F0040EEBEC08F00001C35053
:1007D000D16FC450D26F050EEBEC08F0050EEBECB8
:1007E00008F00001C350D36FC450D46F33EC0DF048
:1007F000FA0E00EC0CF0FA0E00EC0CF0FA0E00EC25
:100800000CF0FA0E00EC0CF020EC09F036EC26F0BF
:1008100061EC0FF075EC0FF0F28EF28CD08E0F01C0
:10082000D89083B6D880D8B01BEF04F00A0E00EC45
:100830000CF00F01D89083B6D880D8B031EF04F017
:100840000F01D89084B2D880D8B02CEF04F00A0EF3
:1008500000EC0CF00F01D89084B2D880D8A053EFF0
:1008600004F0F7EC1FF00201A50EA7633EEF04F0C1
:10087000E70EA8633EEF04F042EF04F016EC35F00B
:100880003CEC0CF000C2E8FF72EC20F00301AD512B
:100890000201A56F54EC0BF0CFEC0AF00101F20E4F
:1008A000066F0CEC0BF00F01D89084B2D880D8A062
:1008B00053EF04F00A0E00EC0CF00F01D89084B254
:1008C000D880D8A053EF04F0809802C5E8FFE8660E
:1008D0008078D2C2E8FFE86673EF04F0808802C532
:1008E000E8FFE866807892981E0EE8CF15F0840E37
:1008F000E8CF14F0800EE8CF13F0D4C217F0E86A06
:10090000E8CF18F027EC12F0D5C2E8FF000113265B
:10091000E86A142213C038F014C039F0040EEBEC6E
:1009200008F0040EEBEC08F00001C350D16FC45086
:10093000D26F050EEBEC08F0050EEBEC08F00001B1
:10094000C350D36FC450D46F0F01D89084B4D880F3
:10095000D8B0B0EF04F00A0E00EC0CF00F01D89004
:1009600084B4D880D8B0C6EF04F00F01D89083B615
:10097000D880D8B0C1EF04F00A0E00EC0CF00F01E3
:10098000D89083B6D880D8A013EF08F00201A0C297
:100990000AF00201FF0E0AB0A56FA56133EF05F062
:1009A0000301A6A113EF05F00F0183BE13EF05F0BD
:1009B000800EB4EC0DF0000EF86E6B0EF76EA20E0A
:1009C000F66E41EC0EF0C00EB4EC0DF0000EF86EB9
:1009D0006B0EF76E420EF66E41EC0EF00F01D890E2
:1009E00084B4D880D8B0FAEF04F00A0E00EC0CF012
:1009F0000F01D89084B4D880D8B0EEEF04F00F0186
:100A0000D89084B4D880D8A0FFEF04F00A0E00EC90
:100A10000CF00F01D89084B4D880D8A0FFEF04F078
:100A2000C80E00EC0CF00201D1B11AEF05F0D1A311
:100A300033EF05F0800E0001A96FBBEC33F0D890C6
:100A4000CFEC28F0D8B02AEF05F00201FF0EA56F19
:100A500033EF05F054EC0BF0CFEC0AF00CEC0BF09C
:100A60000A0E00EC0CF00001010E366EA3C254F029
:100A7000A4C255F00201A25100014F6ECEEC24F049
:100A8000CAEC20F0C00EE8CF90F0E8CF92F0FCAEB8
:100A90004DEF05F00F0193948194000133B06DEF99
:100AA00005F0010E3662D7EF05F00001050EE8CF24
:100AB0005FF0070E93EC0AF0020E366E0001B151A2
:100AC0000201006366EF05F0D7EF05F0006F72ECEE
:100AD00020F0CAEC20F0D7EF05F0010E366E6FEC77
:100AE00024F0B9EC18F098EC07F00201A1A19EEFF8
:100AF00005F00301B651E3EC25F0D8A09EEF05F018
:100B00000201B76796EF05F0B7C075F0B8C076F090
:100B1000B9C077F0BAC078F0BBC079F0BCC07AF049
:100B2000BDC07BF0BEC07CF09EEF05F0F08CF0867F
:100B3000A290E868E8CFFAF0A4EF05F0F09CF08608
:100B4000A280E86AE8CFFAF00201A0B1C7EF05F091
:100B5000EBEC17F0D8B4C7EF05F084EC1AF017EC03
:100B60001AF070EC1CF080EC1DF0E2EC1AF001ECD5
:100B70001BF004EC23F022EC21F00CEC23F0E7EC6A
:100B80001BF00BEC1DF00001F567F8EC10F062ECC7
:100B900003F061EC1EF01AEC0FF00001AE67D5EF28
:100BA00005F00A0EAE6F23EC06F047EF05F0800E5D
:100BB000B4EC0DF0000EF86E6C0EF76ED40EF66EFF
:100BC00041EC0EF0C00EB4EC0DF0000EF86E6B0EA2
:100BD000F76E420EF66E41EC0EF0E6EC1FF0D8A078
:100BE000F4EF05F0B0EC26F0B9EC18F084EC1AF054
:100BF00017EC1AF070EC1CF080EC1DF0E2EC1AF02F
:100C000001EC1BF004EC23F022EC21F00CEC23F0BF
:100C1000E7EC1BF00BEC1DF061EC1EF01AEC0FF092
:100C200047EF05F00001100E0B6EC00EB4EC0DF096
:100C3000000EE16E030EE26EE650A5EC0DF00B2EF9
:100C40001CEF06F012000001840EB4EC0DF0200E33
:100C5000A5EC0DF00201520EA5BF200E0001A5EC7F
:100C60000DF00601CE51E3EC25F0410ED8A0200E88
:100C7000A5EC0DF00301B251E3EC25F04D0ED8B018
:100C80002D0EA5EC0DF00301B351E3EC25F04D0E54
:100C9000D8B02D0EA5EC0DF00301B451E3EC25F016
:100CA0004D0ED8B02D0EA5EC0DF0200EA5EC0DF0DC
:100CB000800EB4EC0DF0B9C20DF0BAC20EF00E6A9F
:100CC0000001640E0F6E000E106E23EC11F013C0C5
:100CD00011F014C012F08DC00DF08EC00EF013C2D2
:100CE0000FF014C210F023EC11F01450E8CF13F001
:100CF0001550E8CF14F0156A010111B190EF06F01C
:100D000000011150135C12501458E8AE90EF06F039
:100D1000C90E00015F6E050E93EC0AF00101116926
:100D20000001D1EC0EF0200EE8CF0AF0300E256461
:100D30000AC025F02550A5EC0DF02650A5EC0DF0CD
:100D40002E0EA5EC0DF02750A5EC0DF00301B651C9
:100D5000E3EC25F0D8A0C9EF06F0A1C2E8FFE81E39
:100D6000E866C0EF06F0800EB4EC0DF0000EF86EF1
:100D70006B0EF76E780EF66E41EC0EF0C9EF06F0D2
:100D8000800EB4EC0DF000C513F001C514F0A7EC13
:100D90000EF00201B8AFE2EF06F0B86B000EE8CF3C
:100DA0000DF0E86AE8CF0EF000C5E8FF26EC0CF085
:100DB000010EE8CF0DF0E86AE8CF0EF001C5E8FFBC
:100DC00026EC0CF0C1EC07F0D8B00CEF07F0D2EC39
:100DD00007F0D8B00CEF07F03BEC26F0D8B00CEFE2
:100DE00007F002EC25F00001AF51E812D8A40CEF97
:100DF00007F00201A0A10AEF07F0C00EB4EC0DF05D
:100E0000000EF86E6B0EF76E5C0EF66E41EC0EF097
:100E10000CEF07F012EC06F0000133B427EF07F0F7
:100E200035A427EF07F03594010E5F6E050E93ECA5
:100E30000AF00001566626EF07F0562ABEC35AF0A4
:100E4000BFC35BF0D66BD76B27EF07F056060001E8
:100E500056A05AEF07F05B665AEF07F03B0E5C6254
:100E600039EF07F0050E5F6E0A0E93EC0AF05AEFA9
:100E700007F01E0E5C6244EF07F0030E5F6E0A0E71
:100E800093EC0AF05AEF07F00A0E5C624FEF07F09E
:100E9000010E5F6E0A0E93EC0AF05AEF07F0060E91
:100EA0005C605AEF07F0010E5F6E0A0E93EC0AF0D9
:100EB0005AEF07F07F0E5C6E5850DA6F5950DB6FB7
:100EC000010E566283EF07F05A505B10D8B472EFF0
:100ED00007F05A50DA6F5B50DB6F000E0301BD6301
:100EE00083EF07F0020E0301BD5DD8B47FEF07F07A
:100EF0000001D651DA6FD751DB6F83EF07F0E86A54
:100F00000001DA6FDB6F00018B0EB4EC0DF0DB51EA
:100F1000E8CF13F0146A156A166A9FEC0EF03A0EC9
:100F2000A5EC0DF0DA51E8CF13F09FEC0EF01200B3
:100F30000301C051E3EC25F0D8A0BEEF07F0030198
:100F4000000EC165BBEF07F000017CBFBEEF07F0EC
:100F50000301C15100010D6E0E6A00010A0E0F6EF1
:100F6000000E106E23EC11F07B51135E7C5114586F
:100F7000D8B0BEEF07F00001F36912000001F36B77
:100F80001200D8900001D8AF1200C00EB4EC0DF0E2
:100F9000000EF86E6C0EF76E0E0EF66E41EC0EF053
:100FA000D88012000D0EEBEC08F00D0EEBEC08F003
:100FB0006BC00DF06CC00EF0A9C20FF0AAC210F009
:100FC00023EC11F000011450136E1550146E1650DE
:100FD000156E166AD1EC0EF00001255026100F0B8D
:100FE000D890D8B41200C00EB4EC0DF0000EF86E1C
:100FF0006B0EF76EFC0EF66E41EC0EF0CB0EB4EC01
:101000000DF000012550A5EC0DF02650A5EC0DF0DB
:101010002E0EA5EC0DF02750A5EC0DF02850A5ECF8
:101020000DF0D88012000F01D89084B4D880D8A0D9
:1010300013EF08F00A0E00EC0CF00F01D89084B406
:10104000D880D8A013EF08F00F01D89083B6D880CD
:10105000D8A024EF08F00A0E00EC0CF00F01D89095
:1010600083B6D880D8A024EF08F0800EB4EC0DF041
:101070000F0183505EEC0EF00F0184505EEC0EF019
:10108000C00EB4EC0DF00F0186505EEC0EF00F01B7
:1010900087505EEC0EF00F01835082868184E8B0A9
:1010A0008296E8B281948098E8B48088320E00EC91
:1010B0000CF00F01D89084B4D880D8B065EF08F058
:1010C0000A0E00EC0CF00F01D89084B4D880D8B090
:1010D00035EF08F00F01D89084B4D880D8A06AEF1B
:1010E00008F00A0E00EC0CF00F01D89084B4D88000
:1010F000D8A06AEF08F0C00EB4EC0DF0000EF86E48
:101100006A0EF76EB20EF66E41EC0EF000010D6A3B
:10111000800EB4EC0DF0000EF86E6A0EF76EE80E5D
:10112000F66E41EC0EF0870EB4EC0DF000010D50A0
:101130006BEC0EF0EBEC08F08C0EB4EC0DF00F0144
:10114000C4CFE8FF6BEC0EF00F01C3CFE8FF6BECF0
:101150000EF0320E00EC0CF00F01D89084B4D88061
:10116000D8B0B8EF08F00A0E00EC0CF00F01D890E0
:1011700084B4D880D8B088EF08F00F01D89084B438
:10118000D880D8A0BDEF08F00A0E00EC0CF00F01DB
:10119000D89084B4D880D8A0BDEF08F000010D2A03
:1011A0000C0E0D6488EF08F035EF08F00001136AAB
:1011B000146A156A166A0A6E0B6A0A50EBEC08F09C
:1011C0000001C3501326C4501422D8B0152A0B2E88
:1011D000DDEF08F012000A6EA10EC06E000EC16EA7
:1011E0000AC0E8FF31EC02F0E8AEC188E89EE844AE
:1011F000E844C26EC2800000C282C2B2FDEF08F0B5
:101200000001C3CF6BF0C4CF6CF00AC0E8FF12003E
:101210000F01C282C2B20AEF09F00001C3506B276E
:10122000C4506C231200EBEC08F008EC09F008EC59
:1012300009F008EC09F000016C336C9F6B3312006D
:1012400000014E6A586A596AD4C2E8FFE8CF57F0E5
:101250000001900E546E010E556E0001900E506EFE
:10126000010E516E526A536A100E0001E8CF4FF022
:101270003A6A3C6A3E6A406A426A446A466A486A16
:101280004A6A4C6A080EE8CF3BF0E8CF3DF0E8CF61
:101290003FF0E8CF41F0E8CF43F0E8CF45F0E8CFAA
:1012A00047F0E8CF49F0E8CF4BF0E8CF4DF0979EFC
:1012B000858E000154500F01E8CFBBFF010155504E
:1012C0000F01E8CFBCFF0A0E0F01E8CFBAFF0F01F4
:1012D000A0800F019E900F01080EE8CFB1FFB180F2
:1012E00012000001FAA1857E0201BAAF7BEF09F07E
:1012F000877083EF09F00001F1B182EF09F0878078
:1013000083EF09F087900001BBCFE8FF5026BCCFE8
:10131000E8FF512250C0E8FFE8CFBBFF51C0E8FF13
:10132000E8CFBCFF0001E86A4E64FCEC09F0000164
:101330004E2A4EC0E8FFFE0B4F60B2EF09F04E6A36
:1013400038C0E8FFE8CF50F052C0E8FF505E39C027
:10135000E8FFE8CF51F053C0E8FF515A526A536A90
:10136000F9EF09F04EA0C7EF09F054C0E8FFE8CF4D
:1013700050F055C0E8FFE8CF51F0BAC2E8FF0001D5
:10138000F1814E62F3EF09F0F191F3EF09F0120EE3
:101390004E62DFEF09F052C0E8FFE8CF50F053C0D3
:1013A000E8FFE8CF51F051325032513250325132D1
:1013B0005032513250320F0E5116F3EF09F0040E35
:1013C000E8CFEAFF000EE8CFE9FF4EC0E8FFE830C3
:1013D000E89EE804E92600EC02F054C0E8FF505E05
:1013E00055C0E8FF515A50C0E8FF522651C0E8FFEF
:1013F00053220F01A19012004FEC0FF059EC0FF0A7
:101400000001010E36620BEF0AF000018286C9B1BD
:101410008296FF0EC96F87900301CDBF13EF0AF0CC
:10142000859E14EF0AF0858E0001572E5BEF0AF0BF
:1014300039EC26F0000156A04AEF0AF00001FF0E39
:10144000F3634AEF0AF05AC0E8FF5B10D8B442EFEA
:101450000AF05A662FEF0AF03C0E5A6E5B065A06E7
:101460005A505C6E0301E86ABD11D8B442EF0AF02D
:1014700000015A505B10D8B442EF0AF0D66BD76B1C
:101480004AEF0AF00001D62B3C0ED6634AEF0AF071
:10149000D66BD72BD4C2E8FFE8CF57F0582A3C0EC2
:1014A00058625BEF0AF0586A592A0501002BD8B43C
:1014B000012B0201B8690201A1A164EF0AF0530EE9
:1014C00081EC0FF00001B46B000183CFE8FF311A0B
:1014D000D8A4306E316E30C0E8FF3212000184CFE4
:1014E000E8FF341AD8A4336E346E33C0E8FF3512E7
:1014F0000001606760076167610762676207AD6747
:10150000AD07AE67AE07AF67AF075E6689EF0AF05B
:1015100012005E2E120080785F4E12005DC0E8FF60
:10152000E8CF5EF01200E8CF5DF0E8CF5EF0D2C207
:10153000E8FFE866A2EF0AF0809802C5E8FFE866D7
:1015400080781200808802C5E8FFE8668078120083
:1015500000010ABEAFEF0AF0819EB0EF0AF0818E63
:10156000828A829A0A460B2EA8EF0AF01200020124
:10157000AD510A6E080E0B6EA8EC0AF00201AC51D8
:101580000A6E080E0B6EA8EC0AF00201AB510A6E4F
:10159000080E0B6EA8EC0AF08686869612000BC128
:1015A00013F00CC114F00DC115F009C117F00AC1F8
:1015B00018F027EC12F00201A55101010F03F350BE
:1015C00000011326D8B0142AD8B0152A0101006BE7
:1015D000016B026B00011350E846E846E880E89290
:1015E0001F0B13B6E88E0101006F0001133614368D
:1015F000153613361436153613361436153613369B
:101600001436153614500101016F000115501F0BDF
:1016100001011009026F1200CFEC0AF0010108511C
:101620000A6E080E0B6EA8EC0AF0010107510A6E53
:10163000080E0B6EA8EC0AF0010106510A6E080EA6
:101640000B6EA8EC0AF086868696010105510A6E9B
:10165000080E0B6EA8EC0AF0010104510A6E080E88
:101660000B6EA8EC0AF0010103510A6E080E0B6E16
:10167000A8EC0AF086868696010102510A6E080ED1
:101680000B6EA8EC0AF0010101510A6E080E0B6EF8
:10169000A8EC0AF0010100510A6E080E0B6EA8ECCE
:1016A0000AF08686869612000F01939E949A939C68
:1016B000819C819E829A989686960201010ED16342
:1016C00081EF0BF004C206F105C207F106C208F172
:1016D00001C203F102C204F103C205F10101700E5F
:1016E0000B6FC60E0C6F000E0D6F0101140E096F0B
:1016F000000E0A6F01010E6B0A0E106F010E0F6FC4
:101700001200020ED163A4EF0BF00AC206F10BC265
:1017100007F10CC208F107C203F108C204F109C2C3
:1017200005F101016C0E0B6FCF0E0C6F000E0D6FEB
:101730000101140E096F000E0A6F01010E6B080EF5
:10174000106F050E0F6F1200030ED163C8EF0BF080
:1017500010C206F111C207F112C208F10DC203F165
:101760000EC204F10FC205F101014A0E0B6F190EF2
:101770000C6F010E0D6F01010A0E096F000E0A6F4A
:1017800001010B0E0E6F320E106F020E0F6F120062
:10179000120087B2E7EF0BF0D5AED9EF0BF0D6CF42
:1017A000CDF0D7CFCEF00001CF2BD8B4D02BF09016
:1017B00012000001CF51D011F090D8A41200E86AB5
:1017C000E8CFD7FFE8CFD6FFD58EF0901200F17AA0
:1017D000F0ACF9EF0BF00301CDA1F5EF0BF0F1AA9E
:1017E000859EF1BA858EF9EF0BF0F1AA858EF1BADC
:1017F000859EF09012000000E82EFBEF0BF0120027
:101800000A6EFA0EFBEC0BF0FA0EFBEC0BF00A2E54
:1018100001EF0CF01200050EE26EE86AE16EE86A74
:10182000AA6EE86AA96EA69EA69CA680A850E66E3F
:10183000A92AF9E112000EC0E8FFAA6E0DC0E8FF68
:10184000A96EA69EA69CA680A8501200A86E0EC0E7
:10185000E8FFAA6E0DC0E8FFA96EA69EA69CA6840E
:10186000F29E550EA76EAA0EA76EA682F28EA1A8B2
:1018700037EF0CF0A1981200800EB4EC0DF0000EC2
:10188000F86E6B0EF76EB40EF66E41EC0EF0C00EF5
:10189000B4EC0DF0000EF86E6B0EF76E300EF66EB7
:1018A00041EC0EF018EC29F0D8A07CEF0CF0C00E43
:1018B000B4EC0DF0000EF86E6B0EF76EC60EF66E01
:1018C00041EC0EF016EC35F00CEC20F00001600E4F
:1018D000AA6F00C2E8FF9DEC20F00201002B03017B
:1018E000072B3A0E076378EF0CF0062B300E076FCC
:1018F0000001AA2F69EF0CF0F7EC1FF000C2E8FF1F
:1019000072EC20F0120000011550F86E1450F76EC2
:101910001350F66E00010E50E26E0D50E16E09009C
:10192000F550E66E0A060900F550E66E0A2E8FEFB6
:101930000CF0120000011550F86E1450F76E1350A1
:10194000F66EA68EA69CA684A688F29E550EA76E5D
:10195000AA0EA76EA6820000F28E0001400E13268A
:10196000000E142215220A2E9AEF0CF0120062ECDF
:1019700003F000011550F86E1450F76E1350F66E18
:10198000A68EA69CA684A688F29E550EA76EAA0EC9
:10199000A76EA682F28E0A0000010E50E26E0D5074
:1019A000E16E400E0B6EE6CFE8FFF56E0F000B2EDA
:1019B000FAD7A68EA69CA684F29E550EA76EAA0EF6
:1019C000A76EA682F28EA6940001400E1326000E8A
:1019D000142215220001400E0D26000E0E220A2EA2
:1019E000B7EF0CF0120000011550F86E1450F76EAE
:1019F0001350F66EA68EA69CA684A688F29E550E5F
:101A0000A76EAA0EA76EA6820000F28E0A00080E2C
:101A10000B6E00010E50E26E0D50E16E080E0C6E62
:101A2000E6CFE8FFF56E0F000C2EFAD7A68EA69C27
:101A3000A684F29E550EA76EAA0EA76EA68200007F
:101A4000F28E0B2EEBD7A6940001400E1326000E4B
:101A5000142215220001400E0D26000E0E220A2E21
:101A6000F3EF0CF012000F019A6A886A9396939A2A
:101A700093988186818A8188140E00EC0CF003C54E
:101A8000E8FFE81EE86671EF0DF0390EB4EC0DF0DA
:101A9000050E00EC0CF0390EB4EC0DF0010E00EC6C
:101AA0000CF0390EB4EC0DF0010E00EC0CF0390E18
:101AB000B4EC0DF01C0EB4EC0DF0520EB4EC0DF0C5
:101AC000690EB4EC0DF0740EB4EC0DF00E0EB4EC27
:101AD0000DF0010EB4EC0DF0060EB4EC0DF092EF2B
:101AE0000DF0380EB4EC0DF0050E00EC0CF0380ED5
:101AF000B4EC0DF0010E00EC0CF0380EB4EC0DF06F
:101B0000010E00EC0CF0380EB4EC0DF0060EB4EC47
:101B10000DF00E0EB4EC0DF0010EB4EC0DF0800ED5
:101B2000B4EC0DF0800EB4EC0DF06A0EF76EC40E3E
:101B3000F66E41EC0EF0C00EB4EC0DF06A0EF76ECE
:101B4000D60EF66E41EC0EF01200C3EC0DF0E6EC92
:101B50000DF0818A8198000000008186000000005D
:101B60008196000000001200C3EC0DF0E6EC0DF0D1
:101B7000819A819800000000818600000000819613
:101B8000000000001200CAEC0DF0D8B0C3EF0DF059
:101B90009A6A12009A688188819A00000000818602
:101BA00000000000D890E8CF41F102C5E8FFE866E8
:101BB000E0EF0DF088BED880819641C1E8FF1200A9
:101BC00088B0D880819641C1E8FF1200886E02C5B6
:101BD000E8FFE81EE866120088CFE8FF886AE8B0F0
:101BE0008888E8B2888AE8B4888CE8B6888EE8B835
:101BF0008886E8BA8884E8BC8882E8BE88801200BB
:101C00001010101010101010181818181818181894
:101C10001C1C1C1C1C1C1C1C1E1E1E1E1E1E1E1EF4
:101C20000101010101010101030303030303030394
:101C300007070707070707070F0F0F0F0F0F0F0FF4
:101C4000800EB4EC0DF00DC0F6FF0EC0F7FFF86A81
:101C500041EC0EF01200C00EB4EC0DF00DC0F6FF1A
:101C60000EC0F7FFF86A41EC0EF01200C00EB4ECA3
:101C70000DF0DAC0F6FFDBC0F7FFF86A41EC0EF0BA
:101C80001200100E44EF0EF00A6E0900F5CFE8FFC7
:101C9000E812D8B45DEF0EF0A5EC0DF00A4E5DEF42
:101CA0000EF00900F5CFE8FFE812D8B45DEF0EF0B2
:101CB000A5EC0DF00A2E45EF0EF012000A6E080E8C
:101CC0000B6E300E0ABE310EA5EC0DF00A360B2E4F
:101CD00061EF0EF012000A6E3A0E0B6E0AC0E8FFBA
:101CE000F00BE842E842E842E84230090B64070F93
:101CF000A5EC0DF00AC0E8FF0F0B30090B64070FCD
:101D0000A5EC0DF00AC0E8FF1200D1EC0EF0255052
:101D1000A5EC0DF02650A5EC0DF02750A5EC0DF02C
:101D20002850A5EC0DF02950A5EC0DF01200D1ECD7
:101D30000EF08AEF0EF0D1EC0EF08DEF0EF0D1EC3C
:101D40000EF090EF0EF0D1EC0EF093EF0EF0D1EC20
:101D50000EF0BBEC0EF02550A5EC0DF02650A5ECD6
:101D60000DF02750A5EC0DF02850A5EC0DF02950F2
:101D7000A5EC0DF012000001300E25621200200EBD
:101D8000256E300E26621200200E266E300E27625F
:101D90001200200E276E300E28621200200E286ED0
:101DA00012000001196A1A6A100E176E270E186EBB
:101DB00027EC12F0300E1310256E1BC013F01CC060
:101DC00014F01DC015F01EC016F0196A1A6AE80E4C
:101DD000176E030E186E27EC12F0300E1310266EDD
:101DE0001BC013F01CC014F01DC015F01EC016F06F
:101DF000196A1A6A640E176E000E186E27EC12F03C
:101E0000300E1310276E1BC013F01CC014F01DC041
:101E100015F01EC016F0196A1A6A0A0E176E000E27
:101E2000186E27EC12F0300E1310286E300E1B10B7
:101E3000296E12000001310E376223EF0FF0F7EC2C
:101E40001FF04DEF0FF0320E37622DEF0FF000C292
:101E5000E8FF72EC20F04DEF0FF0330E376235EFF4
:101E60000FF00CEC20F04DEF0FF0340E37623DEF29
:101E70000FF000C2E8FF9DEC20F0350E37624DEF09
:101E80000FF00001FF0E0D6E030E0E6EE8CF0EF088
:101E9000FF0E26EC0CF04DEF0FF0376A12000F0129
:101EA000ABA21200AB98AB880F01AE500001636B80
:101EB00012000F016BA212006B986B880F016E501D
:101EC00012000C0EE8CFAFFF220EE8CFACFF900E51
:101ED000E8CFABFF0001636B9F9A9D8A1200ACA212
:101EE0006FEF0FF0E8CFADFF1200000EE8CF6FFFED
:101EF000220EE8CF6CFF900EE8CF6BFFA59AA38A65
:101F000012006CA281EF0FF0E8CF6DFF1200E1CF5D
:101F100021F0E2CF22F0000167C0E1FF000166C0BE
:101F2000E2FF6A6BACA292EF0FF0E6CFE8FF000190
:101F30006A27E8CFADFF0001682F92EF0FF021C0B4
:101F4000E1FF22C0E2FF1200E1CF21F0E2CF22F058
:101F5000000167C0E1FF000166C0E2FF6A6B00019B
:101F6000050E606FE86A6065C3EF0FF09EAAB3EFDD
:101F70000FF0AECFE8FFE8CFE6FF00016A270001CF
:101F8000682FAFEF0FF021C0E1FF22C0E2FF120087
:101F90009EAA12000001000E6363DBEF0FF0AECFCC
:101FA000E8FFE8CF64F0550E64631200280EE8CF16
:101FB00061F0632B1200010E6363E5EF0FF0AECF0B
:101FC000E8FFE8CF65F0632B1200020E6363EFEFCA
:101FD0000FF0AECFE8FFE8CF66F0632B1200030EE0
:101FE0006363F9EF0FF0AECFE8FFE8CF67F0632B44
:101FF0001200040E636302EF10F0AECFE8FFE8CFEB
:1020000068F0632B050E63630EEF10F0010E65633D
:102010000CEF10F0A4EC0FF0632B1200060E6363BC
:1020200031EF10F0AECFE8FFE8CF69F0020E656344
:1020300022EF10F087EC0FF06AC0E8FF6FEC0FF0B2
:10204000636B12006AC0E8FF69632CEF10F00C0E9E
:102050006FEC0FF0636B12000D0E6FEC0FF0636B03
:102060001200636B1200A4AA12006ECFE8FF0201F7
:10207000A1B167EF10F0530AD8A412000201A0A189
:10208000120000010F0E7615100981EC0FF075C0DB
:10209000E8FF81EC0FF000010F0E7815200981ECAC
:1020A0000FF0775181EC0FF000010F0E7A15300917
:1020B00081EC0FF0795181EC0FF000010F0E7C15CF
:1020C000400981EC0FF07B5181EC0FF01200000110
:1020D000B4B16EEF10F0B66FB42B1200B56FB42B25
:1020E000020EB46387EF10F0B651F00B100AD8A4BB
:1020F000CCEF10F00F0EB617B6A781EF10F0F00E70
:10210000B613B5C0B7F0B6C0B8F0CCEF10F0040EFF
:10211000B4639EEF10F0B651F00B200AD8A4CCEFB8
:1021200010F00F0EB617B6A798EF10F0F00EB6131A
:10213000B5C0B9F0B6C0BAF0CCEF10F0060EB4637B
:10214000B5EF10F0B651F00B300AD8A4CCEF10F078
:102150000F0EB617B6A7AFEF10F0F00EB613B5C05E
:10216000BBF0B6C0BCF0CCEF10F0080EB463CCEFFF
:1021700010F0B651F00B400AD8A4CCEF10F00F0EBF
:10218000B617B6A7C6EF10F0F00EB613B5C0BDF087
:10219000B6C0BEF0CCEF10F012000C0E0F016F6E47
:1021A000220E6C6E900EE8CF6BFF12000001E80E5D
:1021B0000D26030E0E22780E0D5C070E0E58D8A0C9
:1021C000E5EF10F0EF0EECEF10F00E320D320E32A4
:1021D0000D320E320D320D5081EF0FF0BC0E0D5C42
:1021E000030E0E58D8A0E7EF10F0EF0EECEF10F052
:1021F000F00E81EC0FF0800E81EC0FF075C00DF049
:1022000076C00EF0D6EC10F077C00DF078C00EF06E
:10221000D6EC10F079C00DF07AC00EF0D6EC10F0CC
:102220007BC00DF07CC00EF0EEEC10F07DC00DF028
:102230007EC00EF0EEEC10F07FC00DF080C00EF00E
:10224000EEEC10F0120034EC11F010AE2CEF11F0A7
:102250000D50155E0E50165A0EAE33EF11F00F50A2
:10226000155E1050165A12000001136A146A156A9E
:10227000166A0F500D02F3CF13F0F4CF14F00F5085
:102280000E02F3501426F4501522D8B0162A10501E
:102290000D02F3501426F4501522D8B0162A10500F
:1022A0000E02F3501526F450162212000001246A83
:1022B0001B6A14501310D8B4000C14501718E8BE41
:1022C000241EB06B000E17AE68EF11F0171E172A10
:1022D00014AE6FEF11F0131E141E132A14221450A3
:1022E0001710E8BEFBEF11F017501B5E14361434C4
:1022F0001B3617501B26143614341B36175014B0D7
:102300001B5E14A01B26143614341B36175014B051
:102310001B5E14A01B26143614341B36175014B041
:102320001B5E14A01B26143614341B36175014B031
:102330001B5E14A01B26143614341B36175014B021
:102340001B5E14A01B26143614341B36175014B011
:102350001B5E14A01B26143613341B36175014B002
:102360001B5E14A01B26133613341B36175013B0F4
:102370001B5E13A01B26133613341B36175013B0E5
:102380001B5E13A01B26133613341B36175013B0D5
:102390001B5E13A01B26133613341B36175013B0C5
:1023A0001B5E13A01B26133613341B36175013B0B5
:1023B0001B5E13A01B26133613341B36175013B0A5
:1023C0001B5E13A01B26133613341B36175013B095
:1023D0001B5E13A01B26133613A01B26B0B119EFEA
:1023E00012F024AE000C131E141EE86A132A1422E5
:1023F0001B1E1B2A000C17AE14EF12F014BE10EFB8
:1024000012F0E8CFA9F01350E8CF1BF01B9E133653
:1024100014361450E8CF13F0A951146AF1EF11F0FB
:10242000136A132A146A000C141E131EB02B74EFC7
:1024300011F01B2A17501B62F1EF11F01B6A000EFE
:10244000132A142214AEF1EF11F02388FF0C0001BF
:10245000246A1C6A1B6A155014101310D8B4000C9F
:1024600015501818E8BE241EB06B000E18AE3DEFD4
:1024700012F0171E181E172A182215AE46EF12F07A
:10248000131E141E151E132A14221522155018107F
:10249000E8BED0EF13F017501B5E18501C5A1536CB
:1024A00015341B361C3617501B2618501C221536A7
:1024B00015341B361C36175015A064EF12F01B5E46
:1024C00018501C5A67EF12F01B2618501C221536A4
:1024D00015341B361C36175015A074EF12F01B5E16
:1024E00018501C5A77EF12F01B2618501C22153674
:1024F00015341B361C36175015A084EF12F01B5EE6
:1025000018501C5A87EF12F01B2618501C22153643
:1025100015341B361C36175015A094EF12F01B5EB5
:1025200018501C5A97EF12F01B2618501C22153613
:1025300015341B361C36175015A0A4EF12F01B5E85
:1025400018501C5AA7EF12F01B2618501C221536E3
:1025500015341B361C36175015A0B4EF12F01B5E55
:1025600018501C5AB7EF12F01B2618501C221536B3
:1025700014341B361C36175015A0C4EF12F01B5E26
:1025800018501C5AC7EF12F01B2618501C22143684
:1025900014341B361C36175014A0D4EF12F01B5EF7
:1025A00018501C5AD7EF12F01B2618501C22143654
:1025B00014341B361C36175014A0E4EF12F01B5EC7
:1025C00018501C5AE7EF12F01B2618501C22143624
:1025D00014341B361C36175014A0F4EF12F01B5E97
:1025E00018501C5AF7EF12F01B2618501C221436F4
:1025F00014341B361C36175014A004EF13F01B5E66
:1026000018501C5A07EF13F01B2618501C221436C2
:1026100014341B361C36175014A014EF13F01B5E35
:1026200018501C5A17EF13F01B2618501C22143692
:1026300014341B361C36175014A024EF13F01B5E05
:1026400018501C5A27EF13F01B2618501C22143662
:1026500014341B361C36175014A034EF13F01B5ED5
:1026600018501C5A37EF13F01B2618501C22143632
:1026700013341B361C36175014A044EF13F01B5EA6
:1026800018501C5A47EF13F01B2618501C22133603
:1026900013341B361C36175013A054EF13F01B5E77
:1026A00018501C5A57EF13F01B2618501C221336D3
:1026B00013341B361C36175013A064EF13F01B5E47
:1026C00018501C5A67EF13F01B2618501C221336A3
:1026D00013341B361C36175013A074EF13F01B5E17
:1026E00018501C5A77EF13F01B2618501C22133673
:1026F00013341B361C36175013A084EF13F01B5EE7
:1027000018501C5A87EF13F01B2618501C22133642
:1027100013341B361C36175013A094EF13F01B5EB6
:1027200018501C5A97EF13F01B2618501C22133612
:1027300013341B361C36175013A0A4EF13F01B5E86
:1027400018501C5AA7EF13F01B2618501C221336E2
:1027500013341B361C36175013A0B4EF13F01B5E56
:1027600018501C5AB7EF13F01B2618501C221336B2
:1027700013B0BFEF13F017501B2618501C22B0B136
:10278000F4EF13F024AE000C131E141E151E000EE1
:10279000132A142215221B1E1C1E1B2A1C22000C8D
:1027A00018AEEEEF13F015BEE9EF13F0E8CFA9F085
:1027B0001450E8CF1CF01350E8CF1BF01C9E1436C9
:1027C00015361550E8CF13F0A951156A146AC2EFF7
:1027D00013F0136A132A146A156A000C151E141ECE
:1027E000131EB02B4BEF12F01B2AE86A1C22175065
:1027F0001B62C2EF13F018501C62C2EF13F01C6A88
:102800001B6A000E132A1422152215AEC2EF13F014
:102810002388FF0C1E6A1D6A1C6A1B6A16341B364D
:102820001C361D361E3617501B5E18501C5A195088
:102830001D5A1A501E5AB06AB05B163616341B3633
:102840001C361D361E36B037175016A033EF14F065
:102850001B5E18501C5A19501D5A1A501E5AE86A0D
:10286000B05B3CEF14F01B2618501C2219501D229F
:102870001A501E22E86AB023163616341B361C3650
:102880001D361E36B037175016A052EF14F01B5EDF
:1028900018501C5A19501D5A1A501E5AE86AB05B3B
:1028A0005BEF14F01B2618501C2219501D221A50E1
:1028B0001E22E86AB023163616341B361C361D3627
:1028C0001E36B037175016A071EF14F01B5E18506B
:1028D0001C5A19501D5A1A501E5AE86AB05B7AEFFA
:1028E00014F01B2618501C2219501D221A501E22AB
:1028F000E86AB023163616341B361C361D361E36D3
:10290000B037175016A090EF14F01B5E18501C5AE9
:1029100019501D5A1A501E5AE86AB05B99EF14F00C
:102920001B2618501C2219501D221A501E22E86A1C
:10293000B023163616341B361C361D361E36B037FD
:10294000175016A0AFEF14F01B5E18501C5A195008
:102950001D5A1A501E5AE86AB05BB8EF14F01B26D5
:1029600018501C2219501D221A501E22E86AB0234A
:10297000163616341B361C361D361E36B037175029
:1029800016A0CEEF14F01B5E18501C5A19501D5A99
:102990001A501E5AE86AB05BD7EF14F01B26185085
:1029A0001C2219501D221A501E22E86AB023163626
:1029B00016341B361C361D361E36B037175016A07F
:1029C000EDEF14F01B5E18501C5A19501D5A1A5086
:1029D0001E5AE86AB05BF6EF14F01B2618501C2252
:1029E00019501D221A501E22E86AB02316361534DB
:1029F0001B361C361D361E36B037175016A00CEF8E
:102A000015F01B5E18501C5A19501D5A1A501E5AA8
:102A1000E86AB05B15EF15F01B2618501C22195000
:102A20001D221A501E22E86AB023153615341B36B3
:102A30001C361D361E36B037175015A02BEF15F07B
:102A40001B5E18501C5A19501D5A1A501E5AE86A1B
:102A5000B05B34EF15F01B2618501C2219501D22B4
:102A60001A501E22E86AB023153615341B361C3660
:102A70001D361E36B037175015A04AEF15F01B5EF5
:102A800018501C5A19501D5A1A501E5AE86AB05B49
:102A900053EF15F01B2618501C2219501D221A50F6
:102AA0001E22E86AB023153615341B361C361D3637
:102AB0001E36B037175015A069EF15F01B5E185081
:102AC0001C5A19501D5A1A501E5AE86AB05B72EF10
:102AD00015F01B2618501C2219501D221A501E22B8
:102AE000E86AB023153615341B361C361D361E36E3
:102AF000B037175015A088EF15F01B5E18501C5A00
:102B000019501D5A1A501E5AE86AB05B91EF15F021
:102B10001B2618501C2219501D221A501E22E86A2A
:102B2000B023153615341B361C361D361E36B0370D
:102B3000175015A0A7EF15F01B5E18501C5A19501E
:102B40001D5A1A501E5AE86AB05BB0EF15F01B26EA
:102B500018501C2219501D221A501E22E86AB02358
:102B6000153615341B361C361D361E36B037175039
:102B700015A0C6EF15F01B5E18501C5A19501D5AAF
:102B80001A501E5AE86AB05BCFEF15F01B2618509A
:102B90001C2219501D221A501E22E86AB023153635
:102BA00015341B361C361D361E36B037175015A08F
:102BB000E5EF15F01B5E18501C5A19501D5A1A509B
:102BC0001E5AE86AB05BEEEF15F01B2618501C2267
:102BD00019501D221A501E22E86AB02315361434EB
:102BE0001B361C361D361E36B037175015A004EFA5
:102BF00016F01B5E18501C5A19501D5A1A501E5AB6
:102C0000E86AB05B0DEF16F01B2618501C22195015
:102C10001D221A501E22E86AB023143614341B36C3
:102C20001C361D361E36B037175014A023EF16F091
:102C30001B5E18501C5A19501D5A1A501E5AE86A29
:102C4000B05B2CEF16F01B2618501C2219501D22C9
:102C50001A501E22E86AB023143614341B361C3670
:102C60001D361E36B037175014A042EF16F01B5E0B
:102C700018501C5A19501D5A1A501E5AE86AB05B57
:102C80004BEF16F01B2618501C2219501D221A500B
:102C90001E22E86AB023143614341B361C361D3647
:102CA0001E36B037175014A061EF16F01B5E185097
:102CB0001C5A19501D5A1A501E5AE86AB05B6AEF26
:102CC00016F01B2618501C2219501D221A501E22C5
:102CD000E86AB023143614341B361C361D361E36F3
:102CE000B037175014A080EF16F01B5E18501C5A16
:102CF00019501D5A1A501E5AE86AB05B89EF16F037
:102D00001B2618501C2219501D221A501E22E86A38
:102D1000B023143614341B361C361D361E36B0371D
:102D2000175014A09FEF16F01B5E18501C5A195034
:102D30001D5A1A501E5AE86AB05BA8EF16F01B26FF
:102D400018501C2219501D221A501E22E86AB02366
:102D5000143614341B361C361D361E36B037175049
:102D600014A0BEEF16F01B5E18501C5A19501D5AC5
:102D70001A501E5AE86AB05BC7EF16F01B261850AF
:102D80001C2219501D221A501E22E86AB023143644
:102D900014341B361C361D361E36B037175014A09F
:102DA000DDEF16F01B5E18501C5A19501D5A1A50B0
:102DB0001E5AE86AB05BE6EF16F01B2618501C227C
:102DC00019501D221A501E22E86AB02314361334FB
:102DD0001B361C361D361E36B037175014A0FCEFBC
:102DE00016F01B5E18501C5A19501D5A1A501E5AC4
:102DF000E86AB05B05EF17F01B2618501C2219502B
:102E00001D221A501E22E86AB023133613341B36D3
:102E10001C361D361E36B037175013A01BEF17F0A7
:102E20001B5E18501C5A19501D5A1A501E5AE86A37
:102E3000B05B24EF17F01B2618501C2219501D22DE
:102E40001A501E22E86AB023133613341B361C3680
:102E50001D361E36B037175013A03AEF17F01B5E21
:102E600018501C5A19501D5A1A501E5AE86AB05B65
:102E700043EF17F01B2618501C2219501D221A5020
:102E80001E22E86AB023133613341B361C361D3657
:102E90001E36B037175013A059EF17F01B5E1850AD
:102EA0001C5A19501D5A1A501E5AE86AB05B62EF3C
:102EB00017F01B2618501C2219501D221A501E22D2
:102EC000E86AB023133613341B361C361D361E3603
:102ED000B037175013A078EF17F01B5E18501C5A2C
:102EE00019501D5A1A501E5AE86AB05B81EF17F04C
:102EF0001B2618501C2219501D221A501E22E86A47
:102F0000B023133613341B361C361D361E36B0372D
:102F1000175013A097EF17F01B5E18501C5A19504A
:102F20001D5A1A501E5AE86AB05BA0EF17F01B2614
:102F300018501C2219501D221A501E22E86AB02374
:102F4000133613341B361C361D361E36B037175059
:102F500013A0B6EF17F01B5E18501C5A19501D5ADB
:102F60001A501E5AE86AB05BBFEF17F01B261850C4
:102F70001C2219501D221A501E22E86AB023133653
:102F800013341B361C361D361E36B037175013A0AF
:102F9000D5EF17F01B5E18501C5A19501D5A1A50C5
:102FA0001E5AE86AB05BDEEF17F01B2618501C2291
:102FB00019501D221A501E22E86AB023133613B08E
:102FC000EAEF17F017501B2618501C2219501D222B
:102FD0001A501E22000C0F01D89083B6D880D8B0AA
:102FE000F7EF17F00A0E00EC0CF00F01D89083B643
:102FF000D880D8B06DEF18F00F01D89084B2D88087
:10300000D8B008EF18F00A0E00EC0CF00F01D890C1
:1030100084B2D880D8B06DEF18F00001D8672FEFD8
:1030200018F00001D869030132C30DF033C30EF06C
:103030000001E80E0F6E030E106E23EC11F014C0A9
:103040001CF115C01DF10301345101011C270301BE
:10305000355101011D2334C31AF135C31BF1AAEC0C
:103060002BF0D8B040EF18F0D8A447EF18F00101CA
:103070001A07D8A01B071A07D8A01B0747EF18F09C
:1030800001011A2BD8B41B2B1A2BD8B41B2B1CC133
:103090000DF01DC10EF001011A5100010D5E01017C
:1030A0001B5100010E5A0001000E0F6E010E106E32
:1030B00023EC11F00001E80E176E030E186E27ECDA
:1030C00012F013C032F314C033F31AC134F31BC12E
:1030D00035F301EC1BF0D88412000001D86773EFC0
:1030E00018F0D8941200D86BE7EC20F0D8941200B6
:1030F00000016B51E8CF0DF06C51E8CF0EF06F512D
:103100000D5E70510E5AD8A095EF18F06D51E8CFB2
:103110000FF06E51E8CF10F023EC11F01450E8CF0F
:1031200073F01550E8CF74F012007151E8CF0FF032
:103130007251E8CF10F023EC11F01450E8CF73F087
:103140001550E8CF74F012006BC00DF06CC00EF09B
:103150006F510D5E70510E5A6DC00FF06EC010F0C1
:1031600023EC11F01450E8CF73F01550E8CF74F051
:10317000120085C093F086C094F087C095F088C097
:1031800096F089C097F08AC098F0040EEBEC08F036
:10319000040E13EC09F015C26DF016C26EF017C2E2
:1031A0006FF018C270F019C271F01AC272F078ECA8
:1031B00018F073C034F174C035F173C075F074C089
:1031C00076F0050EEBEC08F0050E13EC09F01BC2CF
:1031D0006DF01CC26EF01DC26FF01EC270F01FC2F7
:1031E00071F020C272F078EC18F073C036F174C040
:1031F00037F173C077F074C078F0060EEBEC08F08E
:10320000060E13EC09F021C26DF022C26EF023C24B
:103210006FF024C270F025C271F026C272F078EC13
:1032200018F073C038F174C039F173C079F074C00C
:103230007AF0070EEBEC08F0070EEBEC08F027C273
:103240006DF028C26EF029C26FF02AC270F0A4ECB3
:1032500018F073C03AF174C03BF173C07BF074C0D6
:103260007CF0030EEBEC08F000010F01C3CFE8FF88
:10327000E8CF8DF0C4CFE8FFE8CF8EF0080EEBEC7E
:1032800008F02DC26FF02EC270F02BC26DF02CC270
:103290006EF0A4EC18F073C085F074C086F0090ECF
:1032A000EBEC08F031C26FF032C270F02FC26DF05B
:1032B00030C26EF0A4EC18F073C087F074C088F0D0
:1032C0000A0EEBEC08F035C26FF036C270F033C274
:1032D0006DF034C26EF0A4EC18F073C089F074C0C5
:1032E0008AF00B0EEBEC08F039C26FF03AC270F0C6
:1032F00037C26DF038C26EF0A4EC18F073C08BF0DA
:1033000074C08CF00301B551E3EC25F0D8A090EF28
:1033100019F00001E80E7D6F030E7E6F95EF19F036
:103320000001180E7D6FFC0E7E6F000EEBEC08F0B6
:103330003BC26DF03CC26EF03DC26FF03EC270F019
:10334000A4EC18F073C07FF074C080F0010EEBECB9
:1033500008F03FC26DF040C26EF041C26FF042C251
:1033600070F0A4EC18F073C081F074C082F0030117
:10337000B751E3EC25F0D8A0C5EF19F00001E80E35
:10338000836F030E846FDFEF19F00301B951E3EC93
:1033900025F0D8A0D3EF19F00001180E836FFC0EB2
:1033A000846FDFEF19F00301B851E3EC25F0D8A0EA
:1033B000DFEF19F00001000E836F000E846F120022
:1033C0000001106A0FBE101E23EC11F00001640E04
:1033D000176E000E186E27EC12F013C011F014C017
:1033E00012F013C00FF014C010F00EAEFDEF19F084
:1033F0000F1E101E0F2AD8B0102A23EC11F0000166
:103400000A0E176E000E186E27EC12F00B50E8CF64
:1034100017F0186A17BE181E27EC12F011500D5E37
:1034200012500E5A13500D2614500E221200030192
:10343000AE51E3EC25F075C00DF076C00EF0D8A0CB
:103440002DEF1AF003011B510001E8CF0FF003012B
:103450001751E8CF0BF035EF1AF003011A510001B4
:10346000E8CF0FF0640EE8CF0BF0E0EC19F00DC0E0
:1034700075F00EC076F00301AF51E3EC25F077C094
:103480000DF078C00EF0D8A051EF1AF003012651CC
:103490000001E8CF0FF003012251E8CF0BF059EF04
:1034A0001AF0030125510001E8CF0FF0640EE8CFB8
:1034B0000BF0E0EC19F00DC077F00EC078F00301CE
:1034C000B051E3EC25F079C00DF07AC00EF0D8A031
:1034D00075EF1AF0030131510001E8CF0FF003013D
:1034E0002D51E8CF0BF07DEF1AF0030130510001B0
:1034F000E8CF0FF0640EE8CF0BF0E0EC19F00DC050
:1035000079F00EC07AF012000301AE51E3EC25F021
:10351000D8A0A3EF1AF075C00FF076C010F017C353
:103520000DF018C30EF00E6A0DBE0E1E23EC11F046
:103530000001640E176E000E186E27EC12F013C017
:1035400075F014C076F00301AF51E3EC25F0D8A07C
:10355000C2EF1AF077C00FF078C010F022C30DF060
:1035600023C30EF00E6A0DBE0E1E23EC11F00001F7
:10357000640E176E000E186E27EC12F013C077F071
:1035800014C078F00301B051E3EC25F0D8A0E1EFCE
:103590001AF079C00FF07AC010F02DC30DF02EC3D1
:1035A0000EF00E6A0DBE0E1E23EC11F00001640E2B
:1035B000176E000E186E27EC12F013C079F014C0CD
:1035C0007AF01200D3C2E8FFE81EE866120000019C
:1035D00086519419E8BEFAEF1AF000018851961945
:1035E000E8BEFAEF1AF000018A519819E8BEFAEF26
:1035F0001AF01200030E00015F6E030E93EC0AF046
:1036000012000201B2519DEC01F00301A75100012B
:103610000F260301A8510001102218C30DF019C391
:103620000EF000010E6AFF0E0DBE0E6E23EC11F0BF
:103630000001640E176E186A196A1A6A27EC12F0F4
:1036400000010301195100010D6E0E6A0DBE0E1E20
:103650000D360E360D5013260E50142213507527BA
:10366000145076230201B3519DEC01F00301A951DE
:1036700000010F260301AA510001102223C30DF0FF
:1036800024C30EF000010E6AFF0E0DBE0E6E23EC79
:1036900011F00001640E176E186A196A1A6A27EC95
:1036A00012F000010301245100010D6E0E6A0DBEDF
:1036B0000E1E0D360E360D5013260E5014221350CA
:1036C0007727145078230201B4519DEC01F00301D7
:1036D000AB5100010F260301AC51000110222EC393
:1036E0000DF02FC30EF000010E6AFF0E0DBE0E6E20
:1036F00023EC11F00001640E176E186A196A1A6A39
:1037000027EC12F0000103012F5100010D6E0E6A2B
:103710000DBE0E1E0D360E360D5013260E50142201
:103720001350792714507A230201B5519DEC01F012
:1037300036C30DF037C30EF000010E6AFF0E0DBE4A
:103740000E6E23EC11F00001640E176E186A196AF0
:103750001A6A27EC12F00301010E3763C7EF1BF062
:103760000001030E0E6E186EE80E0D6E176E7B5183
:103770000D5E7C510E5A196A1A6A13C00FF014C0FC
:1037800010F023EC11F027EC12F0E1EF1BF0020E29
:103790003763E1EF1BF000017B510D6E7C510E6E23
:1037A00013C00FF014C010F023EC11F00001030E51
:1037B000E8CF18F0E80EE8CF17F0196A1A6A27EC7C
:1037C00012F0000113507B2714507C2312000001DB
:1037D0000E6A08C40DF00DBE0E6800010A0E0F6ED1
:1037E000000E106E23EC11F0135075271450762341
:1037F00000010E6A09C40DF00DBE0E6800010A0E2C
:103800000F6E000E106E23EC11F01350772714503A
:10381000782300010E6A0AC40DF00DBE0E68000187
:103820000A0E0F6E000E106E23EC11F01350792764
:1038300014507A2300010E6A0BC40DF00DBE0E6801
:1038400000010A0E0F6E000E106E23EC11F01350E3
:103850007B2714507C2300010E6A0CC40DF00DBEB2
:103860000E6800010A0E0F6E000E106E23EC11F0B0
:1038700013507D2714507E2300010E6A0DC40DF0F5
:103880000DBE0E6800010A0E0F6E000E106E23ECC6
:1038900011F013507F271450802300010E6A0EC4CC
:1038A0000DF00DBE0E6800010A0E0F6E000E106EB8
:1038B00023EC11F0135081271450822300010E6A6B
:1038C0000FC40DF00DBE0E6800010A0E0F6E000E43
:1038D000106E23EC11F01350832714508423120030
:1038E00000010A0E0D6E000E0E6E0301BB51E3ECDB
:1038F00025F0D8A0C1EF1CF003014DAF8EEF1CF0F6
:103900004CC30FF0106A0FBE106823EC11F00001D9
:1039100013C0E8FF752714C0E8FF762303014FAFFB
:10392000A0EF1CF04EC30FF0106A0FBE106823EC1E
:1039300011F0000113C0E8FF772714C0E8FF7823D7
:10394000030151AFB2EF1CF050C30FF0106A0FBE6D
:10395000106823EC11F0000113C0E8FF792714C0B0
:10396000E8FF7A23030153AFC1EF1CF052C30FF0FD
:10397000106A0FBE106823EC11F013C07BF014C066
:103980007CF00301BC51E3EC25F0D8A004EF1DF05E
:10399000030155AFD7EF1CF054C30FF0106A0FBEF0
:1039A000106823EC11F013C075F014C076F0030119
:1039B00057AFE6EF1CF056C30FF0106A0FBE106849
:1039C00023EC11F013C077F014C078F0030159AF65
:1039D000F5EF1CF058C30FF0106A0FBE106823EC0F
:1039E00011F013C079F014C07AF003015BAF04EF5B
:1039F0001DF05AC30FF0106A0FBE106823EC11F0CF
:103A000013C07BF014C07CF000017CAF1200E86AA8
:103A10007B6F7C6F120090C0E8FFC00A32E07DC06F
:103A20000DF07EC00EF000018FC0E8FF0D5E90C06B
:103A3000E8FF0E5A0EBE2FEF1DF019C4E8FF0D5E11
:103A40001AC4E8FF0E5A0EBE41EF1DF0000119C462
:103A5000E8FF8F271AC4E8FF902345EF1DF019C433
:103A6000E8FF0D261AC4E8FF0E220EAE41EF1DF04E
:103A7000000119C4E8FF8F5F1AC4E8FF905B45EFAF
:103A80001DF07DC08FF07EC090F092C0E8FFC00AAC
:103A900032E083C00DF084C00EF0000191C0E8FF59
:103AA0000D5E92C0E8FF0E5A0EBE69EF1DF01BC4FA
:103AB000E8FF0D5E1CC4E8FF0E5A0EBE7BEF1DF042
:103AC00000011BC4E8FF91271CC4E8FF92237FEF8D
:103AD0001DF01BC4E8FF0D261CC4E8FF0E220EAE2D
:103AE0007BEF1DF000011BC4E8FF915F1CC4E8FFE1
:103AF000925B7FEF1DF083C091F084C092F01200C2
:103B00000201A1B112000301B651E3EC25F0D8A0E7
:103B1000120000016267120002019F510001626FF2
:103B20000201010EB6639EEF1DF0010E00015F6EF3
:103B3000050E93EC0AF0280E0001626F75C00DF0BF
:103B400076C00EF041EC1EF0D8A4D4EF1DF00201B7
:103B5000B667ADEF1DF002019E51000176BFBBEFCD
:103B60001DF00301192719AFC5EF1DF0D8A6C5EF49
:103B70001DF0C8EF1DF00301195F19BFC5EF1DF05F
:103B8000D8A6C5EF1DF0CDEF1DF019BFCDEF1DF08C
:103B9000640E1961196FD2EF1DF0640EE81EE82A59
:103BA0001965196FE7EC20F077C00DF078C00EF0C2
:103BB00041EC1EF0D8A40AEF1EF00201B667E3EF55
:103BC0001DF002019E51000178BFF1EF1DF00301CD
:103BD000242724AFFBEF1DF0D8A6FBEF1DF0FEEF6E
:103BE0001DF00301245F24BFFBEF1DF0D8A6FBEFFF
:103BF0001DF003EF1EF024BF03EF1EF0640E2461DE
:103C0000246F08EF1EF0640EE81EE82A2465246F76
:103C1000E7EC20F079C00DF07AC00EF041EC1EF018
:103C2000D8A440EF1EF00201B66719EF1EF00201A2
:103C30009E5100017ABF27EF1EF003012F272FAFFF
:103C400031EF1EF0D8A631EF1EF034EF1EF0030165
:103C50002F5F2FBF31EF1EF0D8A631EF1EF039EFE6
:103C60001EF02FBF39EF1EF0640E2F612F6F3EEF55
:103C70001EF0640EE81EE82A2F652F6FE7EC20F097
:103C8000120000010EAE4AEF1EF00D1E0E1E0D2A90
:103C9000D8B00E2AD8900E320D320E6654EF1EF0B8
:103CA000640E0D6459EF1EF00001640E0D6E000EDF
:103CB0000E6E0D50E832E8321F0BD8740DC0E8FFCD
:103CC00012000001C96B000176BF73EF1EF011C333
:103CD0000DF012C30EF075C00FF076C010F023EC9B
:103CE00011F07DEF1EF015C30DF016C30EF075C078
:103CF0000FF076C010F023EC11F013C30DF014C3D5
:103D00000EF0000114500D2615500E22C7EC1FF0C6
:103D10000DC03EF00EC03FF0000178BF9CEF1EF0DA
:103D20001CC30DF01DC30EF077C00FF078C010F06B
:103D300023EC11F0A6EF1EF020C30DF021C30EF00E
:103D400077C00FF078C010F023EC11F01EC30DF017
:103D50001FC30EF0000114500D2615500E22C7ECA3
:103D60001FF00DC03CF00EC03DF000017ABFC5EF62
:103D70001EF027C30DF028C30EF079C00FF07AC0F3
:103D800010F023EC11F0CFEF1EF02BC30DF02CC37D
:103D90000EF079C00FF07AC010F023EC11F029C3B7
:103DA0000DF02AC30EF0000114500D2615500E22FE
:103DB000C7EC1FF00DC040F00EC041F032C30DF053
:103DC00033C30EF07BC00FF07CC010F023EC11F079
:103DD00034C30DF035C30EF0000114500D261550FC
:103DE0000E22C7EC1FF00DC042F00EC043F03AC3E4
:103DF0000DF03BC30EF08FC00FF090C010F023EC1D
:103E000011F03CC30DF03DC30EF0000114500D261F
:103E100015500E22C7EC1FF00DC044F00EC045F047
:103E200037EF1FF0000180BF22EF1FF01CC30DF021
:103E30001DC30EF07FC00FF080C010F023EC11F016
:103E40002CEF1FF020C30DF021C30EF07FC00FF048
:103E500080C010F023EC11F01EC30DF01FC30EF054
:103E6000000114500D2615500E224AEF1FF03EC3DC
:103E70000DF03FC30EF07FC00FF080C010F023ECB8
:103E800011F040C30DF041C30EF0000114500D2697
:103E900015500E22C7EC1FF00DC046F00EC047F0C3
:103EA00077EF1FF0000182BF62EF1FF011C30DF02A
:103EB00012C30EF081C00FF082C010F023EC11F09D
:103EC0006CEF1FF015C30DF016C30EF081C00FF09C
:103ED00082C010F023EC11F013C30DF014C30EF0E8
:103EE000000114500D2615500E228AEF1FF042C318
:103EF0000DF043C30EF081C00FF082C010F023EC30
:103F000011F044C30DF045C30EF0000114500D260E
:103F100015500E22C7EC1FF00DC048F00EC049F03E
:103F200091C00DF092C00EF00EBE9FEF1FF046C381
:103F30000FF047C310F023EC11F0A5EF1FF04AC3B8
:103F40000FF04BC310F023EC11F048C30DF049C340
:103F50000EF00D5014260E50152214C00DF015C091
:103F60000EF0C7EC1FF00DC04AF00EC04BF0000180
:103F7000D867C6EF1FF00301B151E3EC25F0D8A0DC
:103F8000C6EF1FF038C342F039C343F012000201FC
:103F9000AE5100010D5C0201AF5100010E58E8AEB8
:103FA000D7EF1FF0AEC20DF0AFC20EF0120002014B
:103FB000B05100010D5C0201B15100010E58E8BE84
:103FC0001200B0C20DF0B1C20EF01200000133B405
:103FD000F5EF1FF035A4F5EF1FF03594010E5F6E7D
:103FE000050E93EC0AF0D8801200D8901200000160
:103FF000000E0D6E020E0E6E0001000E136E000E0E
:10400000146E010E156EE86A0A6E83EC0CF0020164
:1040100000510001B16F12000001000E0D6E020E82
:104020000E6E0001000E136E000E146E010E156E62
:10403000040E0A6EB7EC0CF01200E846E8060B6EB0
:104040000001000E0D6E030E0E6E0001000E136EC9
:10405000000E146E010E156E0B501426E86A152220
:10406000100E0A6E83EC0CF01200E846E8060B6EA8
:104070000001000E0D6E080E0E6E0001000E136E94
:10408000000E146E010E156E0B501426E86A1522F0
:10409000400E0A6E83EC0CF00001000EC16F030E9F
:1040A000C26F0001000EBF6F030EC06F0001080E4B
:1040B000C06F100EC36FBBEC24F00001000E0D6E3C
:1040C000080E0E6E0001000E136E000E146E010E2F
:1040D000156E0B501426E86A1522010E0A6EB7EC15
:1040E0000CF01200E846E8060B6E0001000E0D6EA3
:1040F000030E0E6E0001000E136E000E146E010E04
:10410000156E0B501426E86A15220A6E83EC0CF02B
:104110000001000E0D6E040E0E6E0001000E136EF7
:10412000000E146E010E156E0B50E82A1426E86A74
:1041300015220A6E83EC0CF01200E846E8060C6EBD
:104140000001000E0D6E030E0E6E0001000E136EC8
:10415000000E146E010E156E0C501426E86A15221E
:10416000040E0A6EB7EC0CF00001000E0D6E040E8A
:104170000E6E0001000E136E000E146E010E156E11
:104180000C50E82A1426E86A1522040E0A6EB7ECD1
:104190000CF012000001000EC16F030EC26F00018F
:1041A000000EBF6F060EC06F000EC36FBBEC24F095
:1041B0000001000EC16F040EC26F0001000EBF6F40
:1041C000070EC06F000EC36FBBEC24F0120002019B
:1041D0000051E846E8060A6E0001000E0D6E030E5F
:1041E0000E6E0001000E136E000E146E010E156EA1
:1041F0000A501426E86A1522010E0A6EB7EC0CF07C
:10420000120075C099F076C09AF077C09BF078C024
:104210009CF079C09DF07AC09EF07BC09FF07CC07E
:10422000A0F07DC0A1F07EC0A2F07FC0A3F080C04E
:10423000A4F081C0A5F082C0A6F083C0A7F084C01E
:10424000A8F0120001EC21F00301B251E3EC25F0DB
:10425000D8B03DEF21F0030EE26E5C0EE16EDBECB8
:1042600023F0610EE16EDBEC23F0660EE16EDBEC19
:1042700023F06B0EE16EDBEC23F001EC21F0030187
:10428000B351E3EC25F0D8B05EEF21F0030EE26EFF
:10429000700EE16EDBEC23F001EC21F0750EE16EA7
:1042A000DBEC23F001EC21F07A0EE16EDBEC23F085
:1042B00001EC21F07F0EE16EDBEC23F001EC21F04C
:1042C0000301B451E3EC25F0D8B079EF21F0030EEF
:1042D000E26E840EE16EDBEC23F0890EE16EDBEC26
:1042E00023F08E0EE16EDBEC23F0930EE16EDBEC3F
:1042F00023F0120099C00DF09AC00EF010C40FF018
:1043000000010EBE11C40FF0106A0FBE106823EC3E
:1043100011F00001640E176E000E186E27EC12F0FB
:10432000000113C0E8FF9D2714C0E8FF9E239DC035
:104330000DF09EC00EF012C40FF000010EBE13C4AB
:104340000FF0106A0FBE106823EC11F00001640E2C
:10435000176E000E186E27EC12F0000113C0E8FF74
:10436000992714C0E8FF9A239DC00DF09EC00EF05F
:1043700014C40FF000010EBE15C40FF0106A0FBE7A
:10438000106823EC11F00001640E176E000E186E19
:1043900027EC12F0000113C0E8FF9B2714C0E8FFD0
:1043A0009C239FC00DF0A0C00EF016C40FF00001BA
:1043B0000EBE106A0FBE106823EC11F00001640EEF
:1043C000176E000E186E27EC12F0000113C0E8FF04
:1043D0009B2714C0E8FF9C2399C075F09AC076F023
:1043E0009BC077F09CC078F09DC079F09EC07AF0B9
:1043F0009FC07BF0A0C07CF0040117A10EEF22F05B
:104400009BC07FF09CC080F0040118A10EEF22F049
:1044100000017F1F801F7F2BD8B0802B030198A144
:104420002BEF22F09BC00DF09CC00EF09DC00FF052
:104430009EC010F000010DC077F00EC078F00DC0E6
:1044400079F00EC07AF00F50792710507A230F5070
:10445000775F1050785B030199A148EF22F09BC071
:104460000DF09CC00EF099C00FF09AC010F0000142
:104470000DC077F00EC078F00DC075F00EC076F06C
:104480000F507527105076230F50775F1050785BD0
:1044900003019AA103EF23F099C00DF09AC00EF02A
:1044A0000DC075F00EC076F00DC081F00EC082F028
:1044B0000001640E176E000E186E03019C51E81285
:1044C000D8B4ACEF22F0E8BE8AEF22F06408000115
:1044D0000F6E106A76BF7BEF22F075C00DF076C0CC
:1044E0000EF023EC11F027EC12F013C075F014C09D
:1044F00076F0ACEF22F0000181C00DF082C00EF02A
:1045000023EC11F027EC12F013C081F014C082F0FC
:10451000ACEF22F0640F00010F6E106A76AF9FEFD0
:1045200022F075C00DF076C00EF023EC11F027ECF0
:1045300012F013C075F014C076F0ACEF22F0000159
:1045400081C00DF082C00EF023EC11F027EC12F0C8
:1045500013C081F014C082F003019BA1B6EF22F0DA
:104560000001811F821F812BD8B0822B0001640EB5
:10457000176E000E186E03019D51E812D8B403EFB8
:1045800023F00301C651E812D8B4D9EF22F0030199
:10459000C551E3EC25F0D8B003EF23F00001E80E9D
:1045A0000D6E030E0E6E9F510D5EA0510E5AE5EF7B
:1045B00022F00001E80E0D6E030E0E6EA5510D26C1
:1045C000A6510E22D8900E320D329DC30FF09EC31D
:1045D00010F0106A0FBE101E23EC11F027EC12F041
:1045E000135075271450762303019BB1FEEF22F080
:1045F0000001131E141E132AD8B0142A00011350F0
:1046000081271450822312000301A4A1120001EC9F
:1046100021F07AEC21F012000301A4B114EF23F091
:1046200001EC21F07AEC21F003019EA12FEF23F0A1
:104630000301C251E3EC25F0D8A02FEF23F00301D2
:104640009F5100010D6E0E6A00010A0E0F6E000EE2
:10465000106E23EC11F013C07BF014C07CF003014A
:10466000A0A15CEF23F00301C351E3EC25F0D8A037
:104670003EEF23F00301A15147EF23F00301C451A2
:10468000E3EC25F0D8A05CEF23F00301A251000178
:104690000D6E0E6A00010A0E0F6E000E106E23ECF6
:1046A00011F013507B5D14507C59E8AE5CEF23F0A1
:1046B00013C07BF014C07CF012000BC0E8FFF00BBD
:1046C000D8B412000DC06BF00EC06CF00EAE6EEFE1
:1046D00023F00D1E0E1E0D2AD8B00E2A0DC013F0A9
:1046E0000EC014F0640E176E56EC11F000011C6A37
:1046F000090E136086EF23F00BC0E8FFE83AE806E6
:104700000F0BE8B6A3EF23F098EF23F0136E0DC064
:104710001BF00EC01CF0840E00011B5E030E1C5A21
:104720000BC0E8FFE83AE8060F0BE8B6A3EF23F06A
:104730000B0DF350460F1324E8CFD9FF020EE8CF3C
:10474000DAFFADEF23F0E8960B0DF350DA0F1324E8
:10475000E8CFD9FF030EE8CFDAFFDECF0AF0DFCFD4
:104760000BF000010BC00DF00AC0E8FF0D5E0E6AF1
:104770000DBE0E681BC00FF01CC010F023EC11F032
:104780000A0E176E56EC11F00AC0E8FF0A0DF3CFBF
:10479000E8FF1326F4CFE8FF142213C00DF014C075
:1047A0000EF000016CAF120000010D1E0E1E0D2A4E
:1047B000D8B00E2A1200E650E8CF0BF0E812D8B4B9
:1047C000120080EC02F05DEC23F00DC011F00EC081
:1047D00012F0E6CF0AF0E6CFE8FF0001E8CF0DF0D7
:1047E0000E6A0DBE0E1E00010A0E0F6E000E106E38
:1047F00023EC11F011C00DF012C00EF013500D5E3D
:1048000014500E5A0EBE3AEF24F0E6CFE8FF000136
:104810000AAC23EF24F0E8CF13F0E9CF14F00DC079
:1048200011F00EC012F0135080EC02F00DC013F026
:104830000EC014F00A0E176E56EC11F011C00DF0F8
:1048400012C00EF013500F6E106A0FBE101E23EC34
:1048500011F00001640E176E000E186E196A1A6AC4
:1048600027EC12F013C00DF014C00EF00A5000EC4B
:1048700003F01200E6CFE8FFE6CFE8FF00010AAA46
:1048800058EF24F0E8CF13F00DC011F00EC012F075
:10489000135080EC02F00DC013F00EC014F00A0E9D
:1048A000176E56EC11F011C00DF012C00EF013503F
:1048B0000F6E106A0FBE101E23EC11F00001640E83
:1048C000176E000E186E196A1A6A27EC12F013C0E0
:1048D0000DF014C00EF00A5000EC03F012000001BD
:1048E000BD0EC16F030EC26F0001120EBF6F010E2D
:1048F000C06F050EC36FBBEC24F0D90EE8CFD9FF13
:10490000060EE8CFDAFF060EE8CF0CF0DDCFE8FFA9
:10491000E812D8B493EF24F0DFCFE8FFE3EC25F002
:10492000D8B09FEF24F0DDCFE8FF0C2E86EF24F007
:10493000B1C0E8FF02010063A8EF24F01200DECF4F
:10494000E8FFDECFE8FF02010063A8EF24F01200C9
:10495000E8CF00F272EC20F00001120EC16F010EE0
:10496000C26F0001BD0EBF6F030EC06F050EC36F97
:10497000BBEC24F012000001C151E16EC251E26EA5
:104980000001BF51D96EC051DA6EE6CFE8FFE8CF23
:10499000DEFF0001C32FC5EF24F012000001CB6B36
:1049A0000301AE51E3EC25F00001D8B0CB81030147
:1049B000AF51E3EC25F00001D8B0CB830301B05137
:1049C000E3EC25F00001D8B0CB850301B151E3EC55
:1049D00025F00001D8B0CB870301B651E3EC25F0F8
:1049E0000001D8B0CB890301BB51E3EC25F00001F5
:1049F000D8B0CB8B0301BC51E3EC25F00001D8B05B
:104A0000CB8D1200C00EB4EC0DF00301AE51E3ECFF
:104A100025F00001E86AE880CB15D8A01EEF25F04C
:104A2000D8A42FEF25F0CB71000EF86E6C0EF76E48
:104A3000320EF66E41EC0EF0E0EF25F0D8B02FEF1D
:104A400025F0D8B42FEF25F0CB71000EF86E6C0E68
:104A5000F76E200EF66E41EC0EF0E0EF25F003014C
:104A6000AF51E3EC25F00001E86AE882CB15D8A04D
:104A700048EF25F0D8A459EF25F0CB73000EF86E5F
:104A80006C0EF76E560EF66E41EC0EF0E0EF25F070
:104A9000D8B059EF25F0D8B459EF25F0CB73000EFC
:104AA000F86E6C0EF76E440EF66E41EC0EF0E0EF11
:104AB00025F00301B051E3EC25F00001E86AE88439
:104AC000CB15D8A072EF25F0D8A483EF25F0CB75D5
:104AD000000EF86E6C0EF76E7A0EF66E41EC0EF06C
:104AE000E0EF25F0D8B083EF25F0D8B483EF25F0C0
:104AF000CB75000EF86E6C0EF76E680EF66E41EC1C
:104B00000EF0E0EF25F00301B151E3EC25F00001D8
:104B1000D8A099EF25F0CBB79AEF25F0CB77000E10
:104B2000F86E6C0EF76EC20EF66E41EC0EF0E0EF12
:104B300025F0CB970301B651E3EC25F00001D8A096
:104B4000B0EF25F0CBB9B1EF25F0CB79000EF86EC0
:104B50006C0EF76EB00EF66E41EC0EF0E0EF25F045
:104B6000CB990301BB51E3EC25F00001D8A0C7EFBE
:104B700025F0CBBBC8EF25F0CB7B000EF86E6C0E9A
:104B8000F76E8C0EF66E41EC0EF0E0EF25F0CB9B4D
:104B90000301BC51E3EC25F00001D8A0DEEF25F0C5
:104BA000CBBDDFEF25F0CB7D000EF86E6C0EF76EFF
:104BB0009E0EF66E41EC0EF0E0EF25F0CB9D12005C
:104BC000500EAF6F1200E8AA1AEF26F0E8A81AEF0D
:104BD00026F00A6E070BC90FE16E030EE26EE65077
:104BE00000010D6E0E6AE8BE0E6800010A0E0F6E1F
:104BF000000E106E23EC11F00A50070BE846340F3C
:104C0000E16E010EE26EE6CF0DF0E6CF0EF0000190
:104C10000EAE0FEF26F00D1E0E1E0D4A0E2A0DC011
:104C2000E8FF135E0EC0E8FF1458E8360ABE120013
:104C3000D8701200D890E8BA1200D880E8B81200F4
:104C400000011F6E206AE8BC2080070BE82AD8808C
:104C50002036E82E28EF26F030501FB633502014AF
:104C6000D8802062D8901FBED8701200040ED56E76
:104C70001200D59E1200D89087B21200D880D5BEFF
:104C80001200CFC00DF0D0C00EF000013C0E0F6E30
:104C9000000E106E34EC11F013C00DF014C00EF0C5
:104CA0000001240E0F6EF40E106E34EC11F0CDC026
:104CB00017F0CEC018F00001000E196E000E1A6E2B
:104CC0000AEC14F0A5C317F0A6C318F00001186A87
:104CD00027EC12F0C00EB4EC0DF0000EF86E6B0E67
:104CE000F76E900EF66E41EC0EF0CB0EB4EC0DF0BC
:104CF000A7EC0EF0A5C313F0A6C314F0146AC00EFF
:104D0000B4EC0DF0A3EC0EF00001000ECF6F000E1E
:104D1000D06FD88012000001020E3662120000012E
:104D200033A01200FC6A47EF05F0A4EC26F0D8A0EF
:104D30001200FC6A0CEC20F000C2E8FF9DEC20F0B1
:104D4000CAEC20F047EF05F0000130B6AEEF26F0D8
:104D500032A6AEEF26F03296D8801200D89012001C
:104D600000016C0E0E6EE60E0D6EF7EC26F020ECD8
:104D70000EF00001115080EC01F012001EC10DF088
:104D80001FC10EF020EC0EF012000001FB51D8B450
:104D90001200E1CF3EF1E2CF3FF1B9EC18F0000193
:104DA000000E756F000E766F0001000E776F000E1B
:104DB000786F84EC1AF017EC1AF070EC1CF080ECB1
:104DC0001DF001EC1BF004EC23F022EC21F00CECC4
:104DD00023F0E7EC1BF061EC1EF01AEC0FF03EC183
:104DE000E1FF3FC1E2FF12000001FB6912008BEC02
:104DF00026F00001D96BE76BF66BF76BC00EB4ECD5
:104E00000DF00DC0F6FF0EC0F7FFF86A0DC00FF0F1
:104E10000EC010F041EC0EF0FA0E00EC0CF084EC39
:104E20002BF0D8A41AEF27F0110E0D26D8B00E2AB9
:104E300021EF27F0D8A02EEF27F0130E0D26D8B0C3
:104E40000E2A0DC0F6FF0EC0F7FFF86A0900F5CF75
:104E50000DF00900F5CF0EF0FEEF26F095EC26F0F0
:104E6000E6EC1FF0D8A0FEEF26F0150E0D26D8B008
:104E70000E2A0DC0F6FF0EC0F7FFF86A0900F5CF45
:104E800011F00900F5CF12F00FC00DF010C00EF0B8
:104E90000900F5CF0FF00900F5CF10F00900F5CFAC
:104EA000DAF00900F5CFDBF00001C56BC66BC7690E
:104EB0007F0EE8CFC8F012AC6AEF27F00900F5CFFB
:104EC000C5F00900F5CFC6F00900F5CFC7F009001D
:104ED000F5CFC8F012A473EF27F00900F5CFF6F074
:104EE0000900F5CFF7F012A27CEF27F00900F5CF0B
:104EF000F8F00900F5CFF9F012AE81EF27F020ECC1
:104F00000EF012A686EF27F036EC0EF012A2120079
:104F10000001E86AE8CFFBFFF9C0E8FFE8CFFAFF3D
:104F2000F8C0E8FFF96EE8CF0AF00FC01BF010C020
:104F30001CF00FC0F6FF10C0F7FFF86A150EF6263A
:104F4000D8B0F72A0900F5CFE8FF0A62A9EF27F0E9
:104F500012000FC0F6FF10C0F7FF110EF626D8B0F2
:104F6000F72A0900F5CF0FF00900F5CF10F00FC0B8
:104F7000E8FF1B6299EF27F010C0E8FF1C6299EF71
:104F800027F01200000110500F10D8B41200E86A88
:104F9000FB6E1050E8CFFAFF0F50F96E00010F5072
:104FA000E16E1050E26E0001000E1162ECEF27F08E
:104FB0000FC0F6FF10C0F7FFF86A160EF626D8B03D
:104FC000F72ADAC0E1FFDBC0E2FFE7CFE8FF93ECAE
:104FD00027F0F1EC2AF01200010E1162F6EF27F033
:104FE000250EE8CF40F1C7EC29F01200020E116245
:104FF00020EF28F0000112A001EF28F0DA510001A3
:10500000C46FE6CF0AF0E5CF0BF000010AC011F043
:105010000BC012F0129E129C24EC2AF000010FC06B
:10502000E1FF10C0E2FF11C00AF012C00BF00AC08D
:10503000E6FFE7CFE8FFC00B0B120BC0E5FF120045
:10504000030E116235EF28F0E7CFE8FFE83618ECE1
:1050500029F0000ED8B0E81E0A6E00010FC0E1FF73
:1050600010C0E2FF0AC0E7FF1200040E116246EF13
:1050700028F0E7CFE8FF38EC2BF00A6E00010FC0F4
:10508000E1FF10C0E2FF0AC0E7FF1200050E116247
:1050900058EF28F0E7CFE8FF6DEC29F0E8CF0AF0F1
:1050A00000010FC0E1FF10C0E2FF0AC0E7FF1200DD
:1050B000060E11626EEF28F0E7CF0AF00FC0DAF0AB
:1050C00010C0DBF00001A20E0F6E810E106E0AC040
:1050D000E8FF93EC27F0F1EC2AF01200070E1162C2
:1050E00075EF28F0C2EC27F01200080E116286EF6F
:1050F00028F0E7CFE8FF67EC29F0E8CF0AF00001DD
:105100000FC0E1FF10C0E2FF0AC0E7FF0A0E116204
:10511000A7EF28F0E7CFE8FF0001DA15D890D8B460
:10512000D88018EC29F00001DAC00AF000010FC0A5
:10513000E1FF10C0E2FFD8B0A2EF28F00AC0E8FFFC
:10514000E71212000AC0E8FFE81EE71612000B0E75
:105150001162B1EF28F0200EE8CF40F1C7EC29F042
:1051600012000C0E1162CEEF28F0E6CF0AF0E5CF68
:105170000BF000010AC011F00BC012F0A5EC2AF0F0
:1051800000010FC0E1FF10C0E2FF11C00AF012C021
:105190000BF00AC0E6FF0BC0E5FF120012000B6A1D
:1051A000D8B00B1EC00EB4EC0DF0000EF86E6B0EF6
:1051B000F76E300EF66E41EC0EF00BA0F4EF28F017
:1051C000C80EB4EC0DF0280EA5EC0DF0CC0EB4EC2E
:1051D0000DF0290EA5EC0DF0CF0EB4EC0DF0200E65
:1051E000A5EC0DF006EF29F0C80EB4EC0DF0200E82
:1051F000A5EC0DF0CC0EB4EC0DF0280EA5EC0DF0E6
:10520000CF0EB4EC0DF0290EA5EC0DF084EC2BF0D4
:10521000D8B40B6AFF0ED8B00B6E95EC26F0E6EC16
:105220001FF0D8A0DDEF28F0D8900BB0D880120086
:105230000B6AD8B00B1EC80EB4EC0DF0000EF86E61
:105240006B0EF76E6E0EF66E41EC0EF00BA03DEF9E
:1052500029F0C80EB4EC0DF0280EA5EC0DF0CC0E24
:10526000B4EC0DF0290EA5EC0DF0CF0EB4EC0DF062
:10527000200EA5EC0DF04FEF29F0C80EB4EC0DF0A8
:10528000200EA5EC0DF0CC0EB4EC0DF0280EA5EC24
:105290000DF0CF0EB4EC0DF0290EA5EC0DF084EC62
:1052A0002BF0D8B40B6AFF0ED8B00B6E95EC26F03D
:1052B000E6EC1FF0D8A026EF29F0D8900BB0D880EC
:1052C00012000001C765C751C561C5511200000138
:1052D000F4690001A96F71EF29F00001A96F0001C5
:1052E000F46B960E00EC0CF0A9C0E8FF0001136E01
:1052F000146A156A166AD1EC0EF00001F4678FEF9C
:1053000029F0CD0EB4EC0DF02750A5EC0DF028508F
:10531000A5EC0DF02950A5EC0DF09EEF29F0CC0E78
:10532000B4EC0DF02750A5EC0DF02850A5EC0DF0D5
:105330002E0EA5EC0DF02950A5EC0DF0AAEC2BF0EB
:105340000001D8A4AFEF29F0A92BC7C0E8FFA961DD
:10535000A96FA967BCEF29F0A96FBCEF29F0D8A00D
:10536000BCEF29F0A9C0E8FFC561BCEF29F0A9078F
:10537000C5C0E8FFA965A96F95EC26F0E6EC1FF023
:10538000D8A071EF29F00001A9C0E8FF1200C5EC18
:1053900026F0FCC0E8FF7F08E8BEE86AE846E86659
:1053A00000EC0CF0E7CFE8FFE7BEE81EE7BEE82A16
:1053B0000001136E146A156A166AD1EC0EF0CB0E5A
:1053C000B4EC0DF0200EE7BE2D0EA5EC0DF027502D
:1053D000A5EC0DF02850A5EC0DF02950A5EC0DF032
:1053E00040C1E8FFA5EC0DF0AAEC2BF00001D8A419
:1053F000FDEF29F0E72A01EF2AF0D8A001EF2AF00B
:10540000E70695EC26F0E6EC1FF0D8A0C7EF29F0F0
:105410000001FB6B120000011150C75D1250C8590A
:10542000D8B018EF2AF0C751116EC851126E120091
:10543000C551115CC6511258D8B023EF2AF0C5519E
:10544000116EC651126E12000BEC2AF00001CA6BED
:105450000001C451E812D8B436EF2AF0C451E16E0D
:10546000000EE26E11C0E6FF12C0E7FFFCC0E8FFCD
:105470007F08E8BEE86AE846E86600EC0CF011C078
:1054800013F012C014F0D89014321332156A166A51
:10549000D1EC0EF0C90EB4EC0DF02650A5EC0DF0D9
:1054A0002E0EA5EC0DF02750A5EC0DF02850A5EC24
:1054B0000DF02950A5EC0DF06D0EA5EC0DF0530E7E
:1054C000A5EC0DF0AAEC2BF00001D8A477EF2AF0A0
:1054D000112AD8B4122A112AD8B4122AC851126239
:1054E00024EF2AF0C7511160116E24EF2AF0D8A0E2
:1054F00089EF2AF01106D8A012061106D8A01206CC
:10550000C651126224EF2AF0C5511164116E24EFC6
:105510002AF0000133A2CA6933BC94EF2AF00001DB
:10552000A00E116E0F0E126E000133BE9DEF2AF019
:105530000001D00E116E070E126E95EC26F0E6EC0F
:105540001FF0D8A028EF2AF01200FCC0E8FF7F0867
:10555000E8BEE86AE846E86600EC0CF011C013F01B
:1055600012C014F0156A166AD1EC0EF0CB0EB4EC32
:105570000DF02550A5EC0DF02650A5EC0DF02750B0
:10558000A5EC0DF02850A5EC0DF02950A5EC0DF080
:10559000AAEC2BF00001D8A4DAEF2AF0112AD8B433
:1055A000122AC8511262A5EF2AF0C7511160116E7C
:1055B000A5EF2AF0D8A0E9EF2AF01106D8A012062C
:1055C000C6511262A5EF2AF0C5511164116EA5EF04
:1055D0002AF095EC26F0E6EC1FF0D8A0A5EF2AF013
:1055E0001200C00EB4EC0DF00FC0F6FF10C0F7FFB4
:1055F00041EC0EF0FA0E00EC0CF0AAEC2BF0D8A463
:1056000008EF2BF0110E0F26D8B0102A0FEF2BF059
:10561000D8A01CEF2BF0130E0F26D8B0102A0FC005
:10562000F6FF10C0F7FFF86A0900F5CF0FF0090088
:10563000F5CF10F0F1EF2AF095EC26F0E6EC1FF034
:10564000D8A0F1EF2AF0150E0F26D8B0102A0FC0FF
:10565000F6FF10C0F7FFF86A0900F5CF0AF009005D
:10566000F550DAC0E1FFDBC0E2FF0AC0E7FF12003D
:105670000F0BE8B6080B0C0DF3CF13F0F4CF14F0BA
:105680000001D60E1326770E1422CC0EB4EC0DF0CA
:1056900013C0F6FF14C0F7FF41EC0EF0FA0E00EC59
:1056A0000CF0AAEC2BF0D8A45CEF2BF0050E13261F
:1056B000D8B0142A63EF2BF0D8A070EF2BF0070EB0
:1056C0001326D8B0142A13C0F6FF14C0F7FFF86AE7
:1056D0000900F5CF13F00900F5CF14F045EF2BF0DA
:1056E00095EC26F0E6EC1FF0D8A045EF2BF0090E64
:1056F0001326D8B0142A13C0F6FF14C0F7FFF86AB7
:105700000900F5CFE8FF1200040EEBEC08F0040EE0
:10571000EBEC08F0D1C0E8FFC35ED2C0E8FFC45A8A
:10572000C4BE9DEF2BF0640EC35E000EC45AC4BE0F
:10573000A7EF2BF0D884D8901200640EC326000E79
:10574000C422C4AEA7EF2BF0D894D8801200D8940E
:10575000D8901200050EEBEC08F0050EEBEC08F00B
:10576000D3C0E8FFC35ED4C0E8FFC45AC4BEC7EFCD
:105770002BF0640EC35E000EC45AC4BED7EF2BF0EC
:10578000C466C368C3CFFCF0D884D8901200640EFE
:10579000C326000EC422C4AED7EF2BF0C31EC41E16
:1057A000C466C368C3CFFCF0D894D8801200D894E4
:1057B000D8901200E2EF2CF0800EB4EC0DF0000E49
:1057C000F86E6C0EF76EFE0EF66E41EC0EF035EFD5
:1057D0002DF00101160E1E6F6D0E1F6F0101740E6C
:1057E000206F6F0E216F72EC2CF00CEC20F000C2D9
:1057F000E8FF9DEC20F0CAEC20F0120001012E0E13
:105800001E6F6D0E1F6F0101660E206F700E216FEF
:1058100072EC2CF0F5EF2BF00101460E1E6F6D0EB1
:105820001F6F0101500E206F720E216F72EC2CF071
:10583000F5EF2BF001015E0E1E6F6D0E1F6F010163
:10584000420E206F780E216F72EC2CF0F5EF2BF0EA
:105850000101760E1E6F6D0E1F6F0101100E206F7D
:105860007F0E216F72EC2CF0F5EF2BF00001E96B4D
:1058700001018E0E1E6F6D0E1F6F01011A0E206F3B
:10588000850E216F72EC2CF0F5EF2BF00101A60EC6
:105890001E6F6D0E1F6F0101620E206F890E216F4A
:1058A00072EC2CF0F5EF2BF00101BE0E1E6F6D0EA9
:1058B0001F6F0101DC0E206F8C0E216F72EC2CF03B
:1058C000F5EF2BF059EF34F00101EE0E1E6F6D0E67
:1058D0001F6F0101520E206F930E216F72EC2CF09E
:1058E000F5EF2BF0BEEC26F020C10DF021C10EF03B
:1058F000F7EC26F00DC020F10EC021F1F6C026F124
:10590000F7C027F100011150090AD8A4D4EF2CF0F8
:105910000FC00DF010C00EF0F7EC26F00DC022F114
:105920000EC023F1F6C028F1F7C029F10001115093
:10593000090AD8A4BCEF2CF00FC00DF010C00EF077
:10594000F7EC26F00DC024F10EC025F1F6C02AF1C7
:10595000F7C02BF1CEEC27F00001D9B1C2EF2CF04B
:105960002AC10FF02BC110F0C2EC27F024C10DF0BA
:1059700025C10EF0A0EF2CF0CEEC27F00001D9B13C
:10598000D9EF2CF028C10FF029C110F0C2EC27F09C
:1059900020C10DF021C10EF020EC0EF022C10DF05F
:1059A00023C10EF08CEF2CF0CEEC27F00001D9B122
:1059B000120026C10FF027C110F0C2EC27F072EFE1
:1059C0002CF0120000C2E8FF1DEC20F0800EB4ECB9
:1059D0000DF0000EF86E6A0EF76EFA0EF66E41ECE0
:1059E0000EF08D0EB4EC0DF0020100510001136EAB
:1059F000146A156A166A9FEC0EF012EC06F0FCC0F1
:105A0000E8FF7F08E8BEE86AE846E86600EC0CF0CC
:105A1000AAEC2BF0D8A417EF2DF0610E0201002B99
:105A20000063E2EF2CF0010E006FE2EF2CF0D8A043
:105A300025EF2DF002010007000E0063E2EF2CF0CD
:105A4000600E0201006FE2EF2CF0E6EC1FF0D8A030
:105A500008EF2DF000C2E8FF72EC20F000C2E8FF72
:105A6000E8CFB1F00CEC20F01200C00EB4EC0DF059
:105A700012EC06F0000EE16E030EE26E960E00ECE4
:105A80000CF0C00EE124B4EC0DF0E750A5EC0DF0E5
:105A9000C00EE124B4EC0DF00E0EB4EC0DF084EC6D
:105AA0002BF0D8A45DEF2DF0E12A0F0EE1643EEF5C
:105AB0002DF0000EE16E3EEF2DF0D8A069EF2DF035
:105AC000E106FF0EE1623EEF2DF00F0EE16E3EEFBC
:105AD0002DF0AAEC2BF0D8A474EF2DF0E72A7A0E63
:105AE000E760E76E3EEF2DF0D8A07DEF2DF0E706E2
:105AF000200EE764E76E3EEF2DF0E6EC1FF0D8A035
:105B00004FEF2DF00C0EB4EC0DF000C2E8FF9DEC51
:105B100020F012000DC02CF10EC02DF10FC02EF19F
:105B200010C02FF1DCC00DF0DDC00EF00001E80E5A
:105B30000F6E030E106E23EC11F00001000E176EB5
:105B4000010E186E27EC12F013C0DCF014C0DDF06B
:105B50000001DE51DC27DF51DD23E0C00DF0E1C0A4
:105B60000EF00001E80E0F6E030E106E23EC11F024
:105B70000001000E176E010E186E27EC12F0DEC049
:105B8000E0F0DFC0E1F01350E05F1450E15BDCC0F7
:105B90000DF0DDC00EF0C7EC1FF00DC0DCF00EC044
:105BA000DDF0DEC00DF0DFC00EF0C7EC1FF00DC061
:105BB000DEF00EC0DFF0E0C00DF0E1C00EF0C7EC8B
:105BC0001FF00DC0E0F00EC0E1F02CC10DF02DC1B2
:105BD0000EF02EC10FF02FC110F012000DC02CF1ED
:105BE0000EC02DF10FC02EF110C02FF1DCC00DF052
:105BF000DDC00EF00001E80E0F6E030E106E23ECF8
:105C000011F00001000E176E010E186E27EC12F055
:105C1000DEC0DCF0DFC0DDF000011350DC271450E3
:105C2000DD231350DE5F1450DF5BDCC00DF0DDC000
:105C30000EF0C7EC1FF00DC0DCF00EC0DDF0DEC0D2
:105C40000DF0DFC00EF0C7EC1FF00DC0DEF00EC08F
:105C5000DFF02CC10DF02DC10EF02EC10FF02FC1C1
:105C600010F012000DC02CF10EC02DF10FC02EF15E
:105C700010C02FF1DCC00DF0DDC00EF0DE510D5E66
:105C8000DF510E5A0001000E0F6E010E106E23EC54
:105C900011F00001E80E176E030E186E27EC12F0DB
:105CA00013C0DCF014C0DDF0DEC00DF0DFC00EF07C
:105CB000E0510D5EE1510E5A0001000E0F6E010E13
:105CC000106E23EC11F00001E80E176E030E186E33
:105CD00027EC12F013C0E0F014C0E1F02CC10DF07D
:105CE0002DC10EF02EC10FF02FC110F012000DC00B
:105CF0002CF10EC02DF10FC02EF110C02FF1DCC021
:105D00000DF0DDC00EF00001DE510D5EDF510E5AC8
:105D10000001000E0F6E010E106E23EC11F0000159
:105D2000D00E176E070E186E27EC12F013C0DCF0C1
:105D300014C0DDF0DCC00DF0DDC00EF00001E80E97
:105D40000F6E030E106E23EC11F00001000E176EA3
:105D5000010E186E27EC12F000011350DE271450CC
:105D6000DF232CC10DF02DC10EF02EC10FF02FC17D
:105D700010F012000DC02CF10EC02DF10FC02EF14D
:105D800010C02FF10001CAA1F2EF2EF0000E0001A9
:105D90000F18D8B4DDEF2EF0DEC013F0DFC014F022
:105DA000D89013361436DC51135EDD51145A13C0EB
:105DB000E0F014C0E1F0F2EF2EF0000E00010F1839
:105DC000D8B4F2EF2EF0DEC013F0DFC014F0D8909C
:105DD00013361436E051135EE151145A13C0DCF04F
:105DE00014C0DDF02CC10DF02DC10EF02EC10FF04E
:105DF0002FC110F012003E0E0001C46F0001110E01
:105E0000C16F030EC26F0001DC0EBF6F000EC06FCA
:105E10000B0EC36FBBEC24F0E76B8AEC2DF0120085
:105E20003C0E0001C46F00011C0EC16F030EC26F57
:105E300003EF2FF0400E0001C46F0001270EC16F69
:105E4000030EC26F03EF2FF00001110EBF6F030EA0
:105E5000C06FBAEC2EF0E7A1E46B32EC2EF000013B
:105E6000DC0EC16F000EC26F0B0EC36FBBEC24F0D3
:105E70000001C46B120000011C0EBF6F030EC06F47
:105E800029EF2FF00001270EBF6F030EC06F29EF1F
:105E90002FF00DC02CF10EC02DF10FC02EF110C04F
:105EA0002FF1030132C30DF033C30EF00001E80EF1
:105EB0000F6E030E106E23EC11F00001000E176E32
:105EC000010E186E27EC12F013C032F314C033F336
:105ED000030134513227355133232CC10DF02DC12C
:105EE0000EF02EC10FF02FC110F012000DC02CF1DA
:105EF0000EC02DF10FC02EF110C02FF132C30DF0E6
:105F000033C30EF00301345100010D5E030135511E
:105F100000010E5A0001000E0F6E010E106E23ECF0
:105F200011F00001E80E176E030E186E27EC12F048
:105F300013C032F314C033F32CC10DF02DC10EF099
:105F40002EC10FF02FC110F00001C46B1200440EDF
:105F50000001C46F00013A0EC16F030EC26F000151
:105F6000DC0EBF6F000EC06F040EC36FBBEC24F0DD
:105F7000EEEC2DF01200460E0001C46F00013E0E43
:105F8000C16F030EC26FAFEF2FF0480E0001C46F58
:105F90000001420EC16F030EC26FAFEF2FF0000180
:105FA0003A0EBF6F030EC06F77EC2EF00001DC0ECF
:105FB000C16F000EC26F040EC36FBBEC24F0000172
:105FC000C46B120000013E0EBF6F030EC06FD4EF12
:105FD0002FF00001420EBF6F030EC06FD4EF2FF001
:105FE0000001460EC16F030EC26F0001DC0EBF6FD1
:105FF000000EC06F060EC36FBBEC24F08AEC2DF0D0
:10600000120032EC2EF00001DC0EC16F000EC26FE8
:106010000001460EBF6F030EC06F060EC36FBBECD0
:1060200024F00001C46B1200AEC2C5F0AFC2C6F0CE
:10603000B0C2C7F0B1C2C8F0120019C4E8FFE866E8
:1060400028EF30F00401D00E196F070E1A6F1200FE
:10605000E86AE8CF15F00001F40E136E010E146E1D
:1060600019C417F01AC418F027EC12F013C019F471
:1060700014C01AF4E86AE8CF1AF419C4E8FF120051
:106080001BC4E8FFE8664BEF30F00401D00E1B6F35
:10609000070E1C6F1200E86AE8CF15F00001F40E3D
:1060A000136E010E146E1BC417F01CC418F027ECFD
:1060B00012F013C01BF414C01CF4E86AE8CF1CF4FF
:1060C0001BC4E8FF1200DAC0C1F0DBC0C2F000015F
:1060D000E80EBF6F000EC06F050EC36FBBEC24F05F
:1060E000DAC0BFF0DBC0C0F00001E851E83A0F0BA6
:1060F000F06FEF6BE9BFEF1FED6BEB51E9BDED6F9B
:10610000EE6BEC51E9BBEE6F0F0EED17EE17E917D2
:10611000E81712000001F051E83AF00BE813EFBF66
:10612000E98FED51E812D8B499EF30F0ED51EB6FF3
:10613000E98DEE51E812D8B4A1EF30F0EE51EC6FDA
:10614000E98B0001E80EC16F000EC26F050EC36F30
:10615000BBEC24F0120010C4EBF011C4ECF0120000
:10616000EBC010F4ECC011F4120012C4EBF013C435
:10617000ECF01200EBC012F4ECC013F4120014C4E3
:10618000EBF015C4ECF01200EBC014F4ECC015F405
:1061900012000001E7AF12000301196B246B2F6B93
:1061A00012000001E7AF1200A7C313F0A8C314F058
:1061B000855113268651142213C0A7F314C0A8F3E7
:1061C000A9C313F0AAC314F08751132688511422CF
:1061D00013C0A9F314C0AAF3ABC313F0ACC314F0FB
:1061E000895113268A51142213C0ABF314C0ACF3A7
:1061F00012000001E7AF12000301A76BA86BA96BA7
:10620000AA6BAB6BAC6B12000001C56BC52B600EAB
:106210000001C76F12000001E951E96711EF31F089
:106220001200020100C20AF0006F00010AC0E9F08A
:106230009DEC20F00001E9C00AF002010AC000F262
:1062400012000001E7AF120003011951196B18C3C6
:106250000AF000010D6E0E6AE8BE0E680D360E36AD
:106260000001640E0F6E000E106E23EC11F00AC0D8
:1062700017F0186A27EC12F013500301A72700014A
:1062800014500301A82303012451246B23C30AF0F3
:1062900000010D6E0E6AE8BE0E680D360E36000166
:1062A000640E0F6E000E106E23EC11F00AC017F092
:1062B000186A27EC12F013500301A92700011450AB
:1062C0000301AA2303012F512F6B2EC30AF00001F3
:1062D0000D6E0E6AE8BE0E680D360E360001640EB5
:1062E0000F6E000E106E23EC11F00AC017F0186A42
:1062F00027EC12F013500301AB27000114500301E7
:10630000AC2312000001E7AF12002CEC35F01200B4
:10631000BBEC24F012000001DC0EBF6F000EC06F5A
:10632000DAC0C1F0DBC0C2F00B0EC36FBBEC24F0CF
:106330000001DC0EC16F000EC26FDAC0BFF0DBC01F
:10634000C0F00B0EC36F12000201D890A2371200EA
:106350000201D890A23312000001F5AF1200CDEC7B
:1063600010F0120013C20FF014C210F0030E00015F
:10637000AC6F63EC33F00FC013F210C014F21200D4
:10638000A9C20FF0AAC210F00D0E0001AC6F63ECB1
:1063900033F00FC0A9F210C0AAF212000001E7AF5B
:1063A00012000501006B016B0201B86912003CECA0
:1063B0000CF012000001DA51BF6F020EC06FDB510A
:1063C00000011F6E030ED6EC08F014C08DF015C04E
:1063D0008EF0C00EB4EC0DF0000EF86E930EF76E5A
:1063E0002E0EF66E41EC0EF0E6EC1FF0D8A0F4EFA6
:1063F00031F000011F50D6EC08F014C06FF015C04A
:1064000070F014C071F015C072F0FA0E00EC0CF0D0
:10641000C00EB4EC0DF0000EF86E930EF76E400E49
:10642000F66E41EC0EF0E6EC1FF0D8A013EF32F060
:1064300000011F50D6EC08F014C06DF015C06EF0CE
:10644000FA0E00EC0CF000016D516F276E517023B5
:1064500070336F33709F71C017F072C018F0000175
:10646000E80E146E030E156E136A166A6D51175EF0
:106470006E51185A18321732187E196A1A6A27ECA8
:1064800012F013C06DF014C06EF000016D0EC16FFC
:10649000000EC26F040E0001C36FBBEC24F01200AB
:1064A0000001DA51BF6F020EC06FDB5100011F6E99
:1064B000C00EB4EC0DF0000EF86E930EF76E2E0EBB
:1064C000F66E41EC0EF0E6EC1FF0D8A063EF32F070
:1064D00000011F50D6EC08F014C06DF015C06EF02E
:1064E000FA0E00EC0CF0C00EB4EC0DF0000EF86EDD
:1064F000930EF76E400EF66E41EC0EF0E6EC1FF0D8
:10650000D8A07EEF32F000011F50D6EC08F014C086
:106510006FF015C070F0FA0E00EC0CF00001E80E00
:10652000146E030E156E136A166A6DC017F06EC0F6
:1065300018F0196A1A6A00016F51175E7051185AE3
:1065400018AEA4EF32F0FF0E196E1A6E27EC12F09F
:1065500013C06DF014C06EF000016D0EC16F000E1F
:10656000C26F040E0001C36FBBEC24F012000001E7
:10657000DA51BF6F020EC06FDB5100011F6EC00EFB
:10658000B4EC0DF0000EF86E930EF76E1C0EF66E66
:1065900041EC0EF0E6EC1FF0D8A0CAEF32F000019B
:1065A0001F50D6EC08F0000113361436153614C00F
:1065B0006FF015C070F0FA0E00EC0CF0C00EB4ECE9
:1065C0000DF0000EF86E930EF76E2E0EF66E41EC87
:1065D0000EF0E6EC1FF0D8A0E9EF32F000011F50FA
:1065E000D6EC08F0000113361436153614C06DF0E1
:1065F00015C06EF0FA0E00EC0CF0C00EB4EC0DF00D
:10660000000EF86E930EF76E400EF66E41EC0EF033
:10661000E6EC1FF0D8A008EF33F000011F50D6ECD5
:1066200008F0000113361436153614C071F015C089
:1066300072F0FA0E00EC0CF00001E80E146E030E7E
:10664000156E136A166A6DC017F06EC018F0196ADD
:106650001A6A00016F51175E7051185A18AE32EF66
:1066600033F0FF0E196E1A6E27EC12F013C06DF0A6
:1066700014C06EF00001E80E146E030E156E136A5E
:10668000166A6FC017F070C018F0196A1A6A000114
:106690007151175E7251185A18AE50EF33F0FF0E59
:1066A000196E1A6E27EC12F013C071F014C072F05C
:1066B00000016D0EC16F000EC26F060E0001C36FA8
:1066C000BBEC24F01200140E00EC0CF00001AC51F5
:1066D000EBEC08F0C00EB4EC0DF0000EF86E6E0E90
:1066E000F76EAE0EF66E41EC0EF0CB0EB4EC0DF084
:1066F0006BC00DF06CC00EF023EC11F01450136E53
:106700001550146E156AD1EC0EF0200E0A6E300E84
:1067100025640AC025F02550A5EC0DF02650A5EC07
:106720000DF02E0EA5EC0DF02750A5EC0DF0285025
:10673000A5EC0DF0AAEC2BF0D8A4A5EF33F00001E6
:106740000F2AD8B4102A63EF33F0D8A0AFEF33F09C
:1067500000010F06FF0E0F60100663EF33F0E6EC4A
:106760001FF0D8A063EF33F01200FF0EE8CFADF3B7
:1067700054EC0BF012000201FF0EA563CDEF33F0D5
:106780000001A951B4EC0DF0000EF86E6B0EF76E1F
:106790001E0EF66E41EC0EF012000201D1B1EBEFCD
:1067A00033F0D1A3EBEF33F00001A951B4EC0DF0BD
:1067B000000EF86E6B0EF76E0C0EF66E41EC0EF0DE
:1067C0000001A951080FB4EC0DF00201310EA5250E
:1067D000A5EC0DF012000201D1A120EF34F0D1B3ED
:1067E00020EF34F00001A951B4EC0DF0000EF86E6A
:1067F0006B0EF76E7E0EF66E41EC0EF00001A951A5
:106800000E0FB4EC0DF00201300EA525A5EC0DF035
:106810000201A551D890E836500F0001136E146A9A
:10682000156A166AD1EC0EF00001A951040FB4EC00
:106830000DF02850A5EC0DF02950A5EC0DF012003C
:106840000201D1A11200D1A312000001A951B4ECA0
:106850000DF0000EF86E6B0EF76EEA0EF66E41EC60
:106860000EF00001A9510D0FB4EC0DF00201A5517D
:1068700001010E250001136E146A156A166A9FEC59
:106880000EF00201A551D890E836010F0001136EF9
:10689000146A156A166AD1EC0EF00001A951040FB2
:1068A000B4EC0DF02850A5EC0DF02950A5EC0DF03E
:1068B00012000301FF0EAD636EEF34F0C00EB4ECB6
:1068C0000DF0000EF86E6B0EF76E1E0EF66E41ECBC
:1068D0000EF0FA0E00EC0CF07AEF34F00301AD513B
:1068E0000201A56FC00E0001A96FBBEC33F0FA0ED8
:1068F00000EC0CF0AAEC2BF0D8A48AEF34F00101E4
:1069000010510301AD2BAD6359EF34F0FF0EAD6FA5
:1069100059EF34F0D8A09AEF34F00301AD07FE0E22
:10692000AD6359EF34F001011051E8060301AD6F7A
:1069300059EF34F0E6EC1FF0D8A07AEF34F000C243
:10694000E8FF9DEC20F012000DC02CF10EC02DF1DF
:106950000FC02EF110C02FF101C207F202C208F2DF
:1069600003C209F20201033302330133033302335A
:106970000133036B3F0E021701C20DF002C20EF08D
:106980000001140E0F6E000E106E23EC11F013C0F8
:1069900001F214C002F22CC10DF02DC10EF02EC177
:1069A0000FF02FC110F012000DC02CF10EC02DF110
:1069B0000FC02EF110C02FF101C213F002C214F06B
:1069C0000001156A0001050E176E000E186E27EC07
:1069D00012F00201030E0717000E081707C201F29A
:1069E00008C202F209C203F207C20DF208C20EF297
:1069F00009C20FF213C0E8FF0113071314C0E8FF28
:106A000002130813D890000113361436020113C084
:106A1000E8FF0D1314C0E8FF0E132CC10DF02DC1BB
:106A20000EF02EC10FF02FC110F01200000EF86E04
:106A3000930EF76EC80EF66E000E0A6E020EE26E30
:106A4000000EE16E0900F550E66E0A060900F550E9
:106A5000E66E0A2E22EF35F0000EF86E940EF76EF9
:106A6000C80EF66E000E0A6E030EE26E000EE16EA8
:106A70000900F550E66E0A060900F550E66E0A2E8A
:106A800038EF35F0000EF86E950EF76EC80EF66E04
:106A9000000E0A6E040EE26E000EE16E0900F55063
:106AA000E66E0A060900F550E66E0A2E4EEF35F046
:106AB0001200202020202020202020202020202004
:106AC00020200000204D6963726F53746172203280
:106AD000303030200000202056657273696F6E20C0
:106AE000322E306620200000414443204348205885
:106AF00058203D20585858580000202020416972E5
:106B00006372616674202320202000002020202052
:106B10002035332E58204D487A2020200000202098
:106B200020202020204F464620202020202000002A
:106B3000204163636570743F20596573204E6F2058
:106B400000002050726573732020204F7074696FAD
:106B50006E20000020202020202020002020202047
:106B600053747564656E7420202020200000205925
:106B70006573204E6F2000005374646E74002035DE
:106B8000302E5858204D487A202043485820000085
:106B900078426C642052504D203D20787878787887
:106BA00000005265747261637473206172652055D0
:106BB000502100002020466F726D617420466C6188
:106BC0007368202000002020466F726D6174746924
:106BD0006E672E2E2E200000202020436F707969D2
:106BE0006E672E2E2E20202000002037322E58587F
:106BF000204D487A204348585820000052454320F1
:106C0000566F6C74733D2058582E585800005468C5
:106C1000726F74746C65202041646A75737400002F
:106C2000202041494C20442F5220484947482020E9
:106C30000000202041494C20442F5220204C4F5727
:106C4000202000002020454C4520442F5220484958
:106C50004748202000002020454C4520442F52204A
:106C6000204C4F5720200000202052554420442F14
:106C700052204849474820200000202052554420F7
:106C8000442F5220204C4F5720200000202020531A
:106C90004E415020524947485420202000002020D7
:106CA00020534E415020204C4546542020200000C7
:106CB0002020204155544F20205452494D2020205F
:106CC00000002020202020505245534554202020F1
:106CD0002020000020202043414C4942524154458D
:106CE00020202020000053656C65637420204169DA
:106CF00072637261667400FE6C066E0000002041D3
:106D00006972637261667420206E616D6520001681
:106D10006DE66C04000020202020202054696D6561
:106D2000722020202020002E6DFE6C080000202004
:106D300020202020536E617020202020202000463B
:106D40006D166D0C00002020202020536572766F98
:106D5000732020202020005E6D2E6D10000020206A
:106D60002020204D69786572732020202020007635
:106D70006D466D1400002020202020537769746335
:106D8000682020202020008E6D5E6D1800002020DD
:106D900020204F7074696F6E73202020202000A681
:106DA0006D766D1C000020536861726564204F7021
:106DB00074696F6E732000BE6D8E6D200000202000
:106DC00053797374656D205365747570202000D6F7
:106DD0006DA66D24000053656C6563742046726572
:106DE0007175656E637900EE6DBE6D280000202020
:106DF0002020416476616E636564202020200006B7
:106E00006ED66D2C000020202020202045584954AB
:106E100020202020202000E66CEE6D300000456E22
:106E200061626C652020202020202020202000008E
:106E30005265736574203F202020202020202020D0
:106E400000005A65726F20203F2020202020202043
:106E500020200000436C656172203F20202020200C
:106E60002020202000004169726372616674202333
:106E70002020202020200000546F20414654202351
:106E800020202020202020200000426C61646573B7
:106E9000203D202020202020202000004678642053
:106EA0004672737420202020202020200000566F7E
:106EB0006C7473202020202020202020202000001F
:106EC0005769647468202020202020202020202062
:106ED00000004368616E6E656C73202020202020C6
:106EE000202000004E656753686966743F202020AB
:106EF000202020200000506F73203D2020202020E3
:106F000020202020202000004761696E20202020C2
:106F100020202020202020200000496E76657274F9
:106F20003F202020202020202020000054696D6573
:106F3000202873656329202020202020000046722D
:106F400065712C20487A202020202020202000005D
:106F500044656665637420202020202020202020A6
:106F60000000467265712C204B487A20202020209A
:106F7000202000002020202020204D6F646520204C
:106F80002020202000906F047000801E70BD030040
:106F90004D696E75746573202020202020202020EC
:106FA00000B06F746F0540BF0300000000FF0000D9
:106FB0005365636F6E6473202020202020202020E2
:106FC00000D06F906F0540BE0300000000FF00007E
:106FD00020456E61626C6520205377697463682078
:106FE00000EA6FB06F0680C003005468726F74745B
:106FF0006C652020202020202020000470D06F010C
:1070000000C1030045584954202020202020202082
:107010002020202000746FEA6F0300D90000202098
:10702000202055502054696D6572202020200036A4
:10703000704E70000000202020446F776E2054694D
:107040006D6572202020004E701E70010000446F9C
:10705000776E202053746F702054696D6572001E26
:1070600070367002000053522041494C20202020ED
:10707000202020202020008670367201404C030022
:1070800000FF007E0000535220454C452020202068
:1070900020202020202000A670667001404E0300B2
:1070A00000FF007E00005352205255442020202033
:1070B00020202020202000C6708670014050030050
:1070C00000FF007E0000535220544854202020200E
:1070D00020202020202000E670A6700140520300EE
:1070E00000FF007E000053522041494C203F2020E9
:1070F000202020202020000071C67003004D0300D6
:10710000535220454C45203F202020202020202085
:10711000001A71E67003004F030053522052554489
:10712000203F2020202020202020003471007103E7
:1071300000510300535220544854203F2020202067
:1071400020202020004E711A710300530300534C7D
:107150002041494C20202020202020202020006E8B
:10716000713471014054030000FF007E0000534C55
:1071700020454C4520202020202020202020008E4B
:10718000714E71014056030000FF007E0000534C19
:10719000205255442020202020202020202000AEF6
:1071A000716E71014058030000FF007E0000534CD7
:1071B000205448542020202020202020202000CEB1
:1071C000718E7101405A030000FF007E0000534C95
:1071D0002041494C203F202020202020202000E872
:1071E00071AE710300550300534C20454C45203FC0
:1071F0002020202020202020000272CE7103005782
:107200000300534C20525544203F202020202020B2
:107210002020001C72E8710300590300534C2054D5
:107220004854203F202020202020202000367202B9
:107230007203005B03004558495420202020202081
:107240002020202020200066701C720300D900003E
:107250002020202041696C65726F6E202020202044
:107260000070726A73098684730000485EF65D00E0
:1072700020202020456C657661746F7220202020CC
:107280000090725072098684730000765E205E0062
:107290002020202020527564646572202020202048
:1072A00000B0727072098684730000845E345E00E0
:1072B000202020205468726F74746C652020202078
:1072C00000D072907209867A740000EC5E925E00C3
:1072D000202020202020434835202020202020204E
:1072E00000F072B07209866C7500009E5F4E5F0000
:1072F000202020202020434836202020202020202D
:10730000001073D0720986E2750000C45F765F00DA
:10731000202020202020434837202020202020200B
:10732000003073F0720986E2750000D25F8A5F0058
:1073300020202020202043483820202020202020EA
:1073400000507310730986387600000260E05F0019
:1073500020202020537562205472696D73202020F4
:10736000006A7330730980CC760045584954202058
:107370002020202020202020202000507250730345
:1073800000D9000052542F44574E202020202020A6
:107390002020202000A27360740202DC000000287C
:1073A000600043656E74657220202020202020201C
:1073B000202000C07384730202DE000000286000F9
:1073C0004C542F55502020202020202020202020E9
:1073D00000DE73A2730202E0000000286000447522
:1073E000616C20526174652020202020202000F84C
:1073F00073C0730100E200005472696D20202020E8
:107400002020202020202020001274DE730100E3C1
:1074100000004154205253542020202020202020BE
:107420002020002C74F8730300E700004578706F8B
:1074300020484920202020202020202000467412AF
:10744000740100E500004578706F204C4F572020F4
:107450002020202020200060742C740100E6000011
:107460004558495420202020202020202020202062
:1074700000847346740300D90000486967682020BF
:10748000202020202020202020200098740A75022F
:1074900003320342002860004C6F77202020202018
:1074A000202020202020202000B6747A740203348B
:1074B0000342002860005472696D202020202020A3
:1074C00020202020202000D0749874010036030072
:1074D0005472696D204D6F6465202020202020208B
:1074E00000EC74B6740000247537030050726573A5
:1074F000657420202020202020202020000A75D024
:107500007402033803420028600045584954202083
:1075100020202020202020202020007A74EC7403DA
:1075200000D900005472696D204D6F6465204E4F84
:10753000524D414C003C7554750000005472696D09
:10754000204D6F6465202020204C4F570054752437
:10755000750100005472696D204D6F646520202014
:10756000484947480024753C75020000486967682F
:107570002F5570202020202020202020008A75C830
:10758000750202DC0000002860004C6F772F445722
:107590004E20202020202020202000A8756C75027D
:1075A00002DE000000286000204348352020536C94
:1075B000657720526174652000C8758A75088E1938
:1075C000042C6F3A60506000455849542020202018
:1075D0002020202020202020006C75A8750300D9D1
:1075E0000000486967682F55702020202020202047
:1075F00020200000761E760202DC000000286000D9
:107600004C6F772F44574E20202020202020202010
:10761000001E76E2750202DE000000286000455878
:10762000495420202020202020202020202000E25B
:107630007500760300D90000412020202020202062
:107640002020202020202020005676B2760203DC65
:10765000004A0028600042202020202020202020F6
:1076600020202020202000747638760203DE004A95
:1076700000286000432020202020202020202020DF
:107680002020202000927656760203E0004A00284F
:107690006000204348382020536C65772052617485
:1076A000652000B2767476088E1B042C6F8060967D
:1076B00060004558495420202020202020202020F0
:1076C000202000387692760300D9000041696C656D
:1076D000726F6E20202020202020202000EA76BC1F
:1076E00077010208040000E84D00456C657661747E
:1076F0006F722020202020202020000877CC7601E7
:107700000209040000E84D0052756464657220208F
:107710002020202020202020002677EA7601020A5F
:10772000040000E84D005468726F74746C6520208A
:10773000202020202020004477087701020B04003D
:1077400000E84D0043483520202020202020202024
:1077500020202020006277267701020C040000E838
:107760004D004348362020202020202020202020AB
:107770002020008077447701020D040000E84D00CE
:107780004348372020202020202020202020202097
:10779000009E77627701020E040000E84D00434826
:1077A000382020202020202020202020202000BC45
:1077B00077807701020F040000E84D004578697476
:1077C00020202020202020202020202000CC769E59
:1077D000770300D900004E6F6E6500E277367800BF
:1077E00000002041494C00EE77D67701000020458B
:1077F0004C4500FA77E2770200002052554400061B
:1078000078EE7703000020544854001278FA770489
:10781000000020434835001E78067805000020430C
:107820004836002A78127806000020434837003690
:10783000781E780700002043483800D6772A780859
:107840000000202020204D49584552203141202061
:107850002020006278FA7A0986627B5C031461C694
:107860006000202020204D495845522031422020E0
:10787000202000827842780986627B61031461C609
:107880006000202020204D495845522031432020BF
:10789000202000A27862780986627B66031461C6A4
:1078A0006000202020204D4958455220314420209E
:1078B000202000C27882780986627B6B031461C63F
:1078C0006000202020204D49584552203241202080
:1078D000202000E278A2780986627B70031461C6DA
:1078E0006000202020204D4958455220324220205F
:1078F0002020000279C2780986627B75031461C674
:107900006000202020204D4958455220324320203D
:107910002020002279E2780986627B7A031461C60E
:107920006000202020204D4958455220324420201C
:10793000202000427902790986627B7F031461C6A8
:107940006000202020204D495845522033412020FE
:10795000202000627922790986627B84031461C643
:107960006000202020204D495845522033422020DD
:10797000202000827942790986627B89031461C6DE
:107980006000202020204D495845522033432020BC
:10799000202000A27962790986627B8E031461C679
:1079A0006000202020204D4958455220334420209B
:1079B000202000C27982790986627B93031461C614
:1079C000600020202041494C20746F2052554420F3
:1079D000202000E279A2790986147B930360615626
:1079E000610020202052554420746F2041494C20D2
:1079F000202000027AC2790986147B930374616A9D
:107A0000610020202052554420746F20454C4520B1
:107A1000202000227AE2790986147B930388617E14
:107A2000610020202054485420746F20454C45208C
:107A30002020003E7A027A01881604086F00202078
:107A4000202020565441494C202020202020005A3C
:107A50007A227A038898031E6E0020202020204579
:107A60004C45564F4E202020202000767A3E7A0347
:107A70008899031E6E00202020204455414C20414F
:107A8000494C2020202000907A5A7A0980687C0096
:107A9000202020204455414C20454C4520202020CA
:107AA00000AA7A767A0980047D002020202054489C
:107AB0005420484F4C442020202000C47A907A095A
:107AC00080527D002020202049444C4520205550E4
:107AD0002020202000DE7AAA7A0980A07D002020C4
:107AE0004D6978657220206F72646572202000FAFB
:107AF0007AC47A0388A4039C6E0045584954202018
:107B000020202020202020202020004278DE7A0320
:107B100000D90000506F73206761696E202020201B
:107B200020202020002E7B487B0100EB00004E65CA
:107B300067206761696E20202020202020200048D7
:107B40007B147B0100EC0000455849542020202084
:107B5000202020202020202000147B2E7B0300D911
:107B6000000046726F6D2020202020202020202041
:107B70002020007C7B4E7C0400E800005461626C95
:107B800065202020202020202020202000987B62BB
:107B90007B0000087EF00000546F20202020202071
:107BA000202020202020202000B27B7C7B0400E9C4
:107BB00000005265706C6163652020202020202029
:107BC000202000CC7B987B0300EF00005A5020203F
:107BD00020202020202020202020202000E67BB212
:107BE0007B0100EA0000506F73206761696E2020FE
:107BF00020202020202000007CCC7B0100EB000016
:107C0000506F7320496E64202020202020202020E7
:107C1000001A7CE67B0400ED00004E65672067617A
:107C2000696E202020202020202000347C007C0150
:107C300000EC00004E656720496E64202020202063
:107C400020202020004E7C1A7C0400EE00004558C5
:107C500049542020202020202020202020200062A5
:107C60007B347C0300D90000456E61626C65202086
:107C7000202020202020202000827CEA7C03009A03
:107C80000300526576204348372020202020202002
:107C90002020009C7C687C03009B030044494646EE
:107CA00020202020202020202020202000B67C82A0
:107CB0007C01009C0300466C617020202020202065
:107CC00020202020202000D07C9C7C01009D0300EF
:107CD00043524F57202020202020202020202020E9
:107CE00000EA7CB67C0300C60300455849542020B6
:107CF0002020202020202020202000687CD07C0311
:107D000000D90000456E61626C6520202020202093
:107D100020202020001E7D387D03001704005265BE
:107D200076204348362020202020202020200038A4
:107D30007D047D030018040045584954202020206C
:107D4000202020202020202000047D1E7D0300D93B
:107D50000000456E61626C652020202020202020DC
:107D60002020006C7D867D03009E0300506F7369A8
:107D700074696F6E202020202020202000867D52F4
:107D80007D01009F030045584954202020202020D9
:107D900020202020202000527D6C7D0300D900008F
:107DA000456E61626C65202020202020202020204C
:107DB00000BA7DEE7D0300A00300506F7369746903
:107DC0006F6E204120202020202000D47DA07D0146
:107DD00000A10300506F736974696F6E2042202008
:107DE0002020202000EE7DBA7D0100A2030045582E
:107DF000495420202020202020202020202000A0C6
:107E00007DD47D0300D900005461626C6520202080
:107E1000202020204E6F6E6500207EF87E0000003E
:107E20004169726372616674205461626C652031CD
:107E300000387E087E0900004169726372616674D1
:107E4000205461626C65203200507E207E0A000062
:107E5000476C6F6162616C205461626C65202031F7
:107E600000687E387E010000476C6F6162616C20A3
:107E70005461626C6520203200807E507E020000DA
:107E8000476C6F6162616C205461626C65202033C5
:107E900000987E687E030000476C6F6162616C2011
:107EA0005461626C6520203400B07E807E04000046
:107EB000476C6F6162616C205461626C6520203593
:107EC00000C87E987E050000476C6F6162616C207F
:107ED0005461626C6520203600E07EB07E060000B2
:107EE000476C6F6162616C205461626C6520203761
:107EF00000F87EC87E070000476C6F6162616C20ED
:107F00005461626C6520203800087EE07E08000025
:107F1000202020202041494C204452202020202095
:107F2000002A7FFE800680AE03002020202020450E
:107F30004C45204452202020202000447F107F0602
:107F400080AF03002020202020525544204452209E
:107F500020202020005E7F2A7F0680B003002020A2
:107F600020202050524553455420202020200078C6
:107F70007F447F0680B10300202020204D495845D2
:107F8000522020312020202000927F5E7F0680B288
:107F90000300202020204D49584552202032202027
:107FA000202000AC7F787F0680B3030020202020B3
:107FB0004D495845522020332020202000C67F9272
:107FC0007F0680B403002020202020204348352055
:107FD00020202020202000E07FAC7F0680B5030019
:107FE000202020204155544F205452494D2020201C
:107FF00000FA7FC67F0680B60300202020202043A1
:1080000048382041202020202020001480E07F06D6
:1080100080B7030020202020204348382042202021
:1080200020202020002E80FA7F0680B80300202028
:1080300020202043483820432020202020200048B2
:108040008014800680B9030020202020534E415028
:1080500020205220202020200062802E800680BB1D
:10806000030020202020534E415020204C2020206F
:108070002020007C8048800680BC03002054687269
:108080006F74746C652020486F6C64200096806269
:10809000800680C2030020202049646C6520557052
:1080A00020203120202000B0807C800680C3030087
:1080B00020202049646C652055702020322020202B
:1080C00000CA8096800680C4030020202020202043
:1080D00043524F5720202020202000E480B080060B
:1080E00080C50300205472696767657220506F690C
:1080F0006E74732000FE80CA800980188100455884
:108100004954202020202020202020202020001042
:108110007FE4800300D9000041696C65726F6E20B6
:108120005472696720506F7300348188810188C957
:1081300003F66E00456C657661746F722054726749
:1081400020506F7300508118810188CA03F66E00B9
:1081500052756464657220205472696720506F7391
:10816000006C8134810188CB03F66E005468726F15
:1081700074746C652054726720506F73008881504E
:10818000810188CC03F66E004558495420202020F8
:1081900020202020202020200018816C810300D97D
:1081A0000000202020202020204F4E2020202020B2
:1081B000202000BA810285100000202020202020ED
:1081C000204F464620202020202000D281A281205E
:1081D0000000535741202020202020202020202054
:1081E0004F4E00EA81BA8100000053574120202001
:1081F000202020202020204F4646000282D281806D
:108200000000535742202020202020202020202022
:108210004F4E001A82EA810100005357422020206D
:10822000202020202020204F4646003282028281DA
:1082300000005357432020202020202020202020F1
:108240004F4E004A821A82020000535743202020DA
:10825000202020202020204F464600628232828249
:108260000000535744202020202020202050524539
:108270005353007A824A82830000535744202020BF
:1082800020202052454C4541534500928262820392
:10829000000053574520202020202020202020208F
:1082A0004F4E00AA827A82040000535745202020B6
:1082B000202020202020204F464600C28292828427
:1082C000000053574620202020202020202020205E
:1082D0004F4E00DA82AA8205000053574620202024
:1082E000202020202020204F464600F282C2828596
:1082F000000053574720202020202020202020202D
:108300004F4E000A83DA8206000053574720202090
:10831000202020202020204F4646002283F2828603
:1083200000005357482020202020202020202020FB
:108330004F4E003A830A83070000535748202020FD
:10834000202020202020204F464600528322838771
:108350000000535749202020202020202050524543
:108360005353006A833A83890000535749202020E1
:1083700020202052454C45415345008283528309B9
:10838000000053574A202020202020202020202099
:108390002041009A836A838B000053574A20202093
:1083A0002020202020202020204200B28382834BE6
:1083B000000053574A202020202020202020202069
:1083C000204300CA839A838C000053574B202020FF
:1083D00020202020202020204F4E00E283B2830D59
:1083E000000053574B202020202020202020204F09
:1083F000464600FA83CA838D000053574C20202044
:1084000020202020205052455353001284E2838EB6
:10841000000053574C20202020202052454C45413D
:108420005345002A84FA830E000053574D20202024
:108430002020202020505245535300428412848F24
:10844000000053574D20202020202052454C45410C
:108450005345005A842A840F000041696C65726F8D
:108460006E202020202020204F4E00728442843035
:10847000000041696C65726F6E2020202020204F23
:108480004646008A845A84B00000456C6576617463
:108490006F722020202020204F4E00A28472843151
:1084A0000000456C657661746F7220202020204F9B
:1084B000464600BA848A84B10000527564646572CD
:1084C00020202020202020204F4E00D284A2843261
:1084D0000000527564646572202020202020204F07
:1084E000464600EA84BA84B200005468726F74741D
:1084F0006C652020202020204F4E000285D284333E
:1085000000005468726F74746C6520202020204F26
:10851000464600A281EA84B3000020202041757401
:108520006F20205472696D2020200034853E86091A
:1085300080CE87005265736574204175746F205436
:1085400072696D730052851A85038CE700306E9254
:1085500061002020205472696D20205A65726F20BE
:1085600020200070853485038CE700426EA26100F4
:10857000436C656172205472696D205A65726F7325
:10858000008E855285038CE700546EF26100204115
:108590006C7420202041697263726166742000A8A7
:1085A000857085098058860020436F7079202041AE
:1085B000697263726166742000C8858E85058EE9D4
:1085C00000786E16620862002020536574204465AE
:1085D0006661756C7473202000E685A885038CE7BE
:1085E00000306E0463004E756D202070726F702035
:1085F000626C61646573000686C88505C8A5038A38
:108600006E01000500005265747261637473205737
:1086100061726E696E67002286E6850388A6031E76
:108620006E00204155584F555420436F6E74726F41
:108630006C20003E86068600808A88BA0200455873
:108640004954202020202020202020202020001AF3
:108650008522860300D9000020416C74202331203C
:108660002020202020202020007886B4870540CFBD
:10867000030000000060000020416C7420202331C2
:10868000205377697463682000928658860680CEEE
:10869000030020416C742023322020202020202041
:1086A000202000B28678860540D1030000000060DB
:1086B000000020416C7420202332205377697463BA
:1086C000682000CC8692860680D0030020416C741E
:1086D00020233320202020202020202000EC86B2E0
:1086E000860540D3030000000060000020416C7448
:1086F000202023332053776974636820000687CCD9
:10870000860680D2030020416C7420233420202070
:10871000202020202020002687EC860540D503005D
:1087200000000060000020416C742020233420539E
:1087300077697463682000408706870680D4030049
:1087400020416C7420233520202020202020202050
:1087500000608726870540D7030000000060000006
:1087600020416C742020233520537769746368207E
:10877000007A8740870680D6030020416C7420234E
:1087800036202020202020202020009A8760870586
:1087900040D9030000000060000020416C742020DC
:1087A0002336205377697463682000B4877A87067C
:1087B00080D8030045584954202020202020202024
:1087C000202020200058869A870300D900004154B9
:1087D000206D6F646520202020202020202000EACA
:1087E000873C8800005688B60200415420737465A7
:1087F00070202020202020202020000488CE870503
:10880000009E02004154207469636B732020202075
:1088100020202020001E88EA8705009F0200746F38
:1088200020545A2020202020202020202020003CDE
:108830008804880304E70000004262004558495458
:1088400020202020202020202020202000CE871E35
:10885000880300D900004154206D6F6465202020FA
:10886000202020496E6300708870880000B60200E6
:108870004154206D6F6465204F6E652053686F749E
:1088800000568856880100B60200202020202020B3
:108890002043483120202020202000A2884A89013E
:1088A00000002020202020202043483220202020AB
:1088B000202000BA888A8803000020202020202061
:1088C0002043483320202020202000D288A2880581
:1088D0000000202020202020204348342020202079
:1088E000202000EA88BA88070000202020202020CD
:1088F00020434835202020202020000289D28809EA
:108900000000202020202020204348362020202046
:108910002020001A89EA880B000020202020202037
:108920002043483720202020202000328902890D52
:108930000000202020202020204348382020202014
:108940002020004A891A890F0000202020202020A2
:108950002050504D202020202020008A88328980FD
:10896000000020202042756464792020426F782026
:108970002020007C8996890980B089002020202051
:10898000205461626C65732020202020009689624B
:108990008909804A8A0045584954202020202020F7
:1089A0002020202020200062897C890300D900003B
:1089B0004D6173746572203F2020202020202020EC
:1089C00000CA89008A0300A1020020204D6173744F
:1089D000657220204D6F6465202000E689B0890013
:1089E000001A8AB7020053747564656E74203F20C4
:1089F00020202020202000008ACA890300A0020035
:108A000045584954202020202020202020202020AC
:108A100000B089E6890300D900004D204D6F6465E0
:108A20003D4D6963726F5374617200328A328A00FD
:108A300000004D204D6F64653D4675746162612094
:108A40002020001A8A1A8A0100004169726372614B
:108A50006674205461626C652031006A8A8A8B09D1
:108A600086A48BDA03106316630041697263726136
:108A70006674205461626C652032008A8A4A8A09D1
:108A800086A48BE5031063166300476C6F62616C0C
:108A900020205461626C6520203100AA8A6A8A090C
:108AA00086A48B46021063166300476C6F62616C8C
:108AB00020205461626C6520203200CA8A8A8A09AB
:108AC00086A48B51021063166300476C6F62616C61
:108AD00020205461626C6520203300EA8AAA8A094A
:108AE00086A48B5C021063166300476C6F62616C36
:108AF00020205461626C65202034000A8BCA8A09E8
:108B000086A48B67021063166300476C6F62616C0A
:108B100020205461626C65202035002A8BEA8A0986
:108B200086A48B72021063166300476C6F62616CDF
:108B300020205461626C65202036004A8B0A8B0924
:108B400086A48B7D021063166300476C6F62616CB4
:108B500020205461626C65202037006A8B2A8B09C3
:108B600086A48B88021063166300476C6F62616C89
:108B700020205461626C65202038008A8B4A8B0962
:108B800086A48B9302106316630045584954202035
:108B900020202020202020202020004A8A6A8B03C9
:108BA00000D90000504F53203020202020202020CA
:108BB0002020202000BE8BC28C0100DC0000504F22
:108BC000532031202020202020202020202000D8C9
:108BD0008BA48B0100DD0000504F53203220202059
:108BE000202020202020202000F28BBE8B0100DEE0
:108BF0000000504F53203320202020202020202010
:108C00002020000C8CD88B0100DF0000504F532037
:108C100034202020202020202020202000268CF21C
:108C20008B0100E00000504F5320352020202020F1
:108C300020202020202000408C0C8C0100E100002E
:108C4000504F53203620202020202020202020207C
:108C5000005A8C268C0100E20000504F5320372030
:108C60002020202020202020202000748C408C01F7
:108C700000E30000504F53203820202020202020E7
:108C800020202020008E8C5A8C0100E40000504FE0
:108C9000532039202020202020202020202000A820
:108CA0008C748C0100E50000504F5320313020209F
:108CB000202020202020202000C28C8E8C0100E665
:108CC000000045584954202020202020202020202A
:108CD000202000A48BA88C0300D900002054582029
:108CE000566F6C7420204D657465722000F88CB44A
:108CF0008E07886463AE6E00545820416C61726DBB
:108D000020566F6C7461676500188DDC8C08C8B9DB
:108D100002AE6E0000FF0000526573657420426170
:108D200074742054696D657200368DF88C038CE77D
:108D300000306E9C630020525820566F6C742020C7
:108D40004D657465722000528D188D07888063AE62
:108D50006E00536572766F20204D696E2050756CE1
:108D6000736500728D368D02C8AE02C06EE803884E
:108D70001300536572766F20204D61782050756C1A
:108D8000736500928D528D02C8B002C06EE80388F0
:108D900013004E756D62657220204368616E6E65CA
:108DA0006C7300B68D728D05CEA202D26E040009DE
:108DB00000486350630020202053796E6320776958
:108DC00064746820202000D68D928D02C8A302C052
:108DD0006EC800DC05002020536869667420496E67
:108DE00076657274202000F28DB68D0388CD03E481
:108DF0006E002020466F726D617420466C6173684E
:108E00002020000C8ED68D0780AE6300202020200D
:108E1000436F6E66696775726520202000268EF2AA
:108E20008D09802E8F0020204A6F79537469636BFF
:108E30002043616C202000408E0C8E0980EA910056
:108E400020202020202020464D532020202020209C
:108E5000005E8E268E038CF5001E6E586300204641
:108E600072657175656E63792042616E6420007C65
:108E70008E408E0084CE8ED1026A67002042757AC1
:108E80007A65722020496E766572742000988E5E35
:108E90008E0388D2021A6F005472696D2043656E8A
:108EA000746572204265657000B48E7C8E0388D331
:108EB000021E6E00455849542020202020202020EA
:108EC0002020202000DC8C988E0300D90000202078
:108ED0002020204E6F20205246202020202000E617
:108EE0008E168F0000002020202020353020204DBD
:108EF000487A2020202000FE8ECE8E010000202007
:108F0000202020353320204D487A202020200016B4
:108F10008FE68E0200002020202020373220204DB6
:108F2000487A2020202000CE8EFE8E0300004F7550
:108F300074707574206368616E6E656C2031004AD0
:108F40008F7E90000198900004004F7574707574C6
:108F5000206368616E6E656C203200668F2E8F0014
:108F60000198900104004F757470757420636861F6
:108F70006E6E656C203300828F4A8F0001989002DC
:108F800004004F7574707574206368616E6E656C53
:108F90002034009E8F668F000198900304004F7567
:108FA00074707574206368616E6E656C203500BAEC
:108FB0008F828F000198900404004F75747075744F
:108FC000206368616E6E656C203600D68F9E8F00C0
:108FD0000198900504004F75747075742063686182
:108FE0006E6E656C203700F28FBA8F000198900684
:108FF00004004F7574707574206368616E6E656CE3
:109000002038000E90D68F00019890070400536519
:109010006C6563742041696C20205472696D002A6C
:1090200090F28F00016891B2020053656C65637421
:1090300020456C6520205472696D0046900E9000AA
:10904000016891B3020053656C65637420527564C6
:1090500020205472696D0062902A9000016891B4DA
:10906000020053656C656374205468742020547248
:10907000696D007E90469000016891B502004558E8
:109080004954202020202020202020202020002E95
:109090008F62900300D900002020202041696C6578
:1090A000726F6E202020202000B2904E910100E8C7
:1090B000000020202020456C657661746F722020AE
:1090C000202000CC9098900200E800002020202072
:1090D00020527564646572202020202000E690B242
:1090E000900300E80000202020205468726F747400
:1090F0006C6520202020000091CC900400E8000046
:1091000020202020202020434835202020202020FF
:10911000001A91E6900500E8000020202020202081
:109120002043483620202020202000349100910642
:1091300000E8000020202020202020434837202065
:1091400020202020004E911A910700E800002020E6
:109150002020202020434838202020202020009854
:109160009034910800E80000202020204E6F20203D
:109170005472696D20202020008291D0910000E877
:10918000000020202020205472696D2031202020F2
:109190002020009C9168910100E800002020202000
:1091A000205472696D2032202020202000B6918248
:1091B000910200E8000020202020205472696D20D8
:1091C00033202020202000D0919C910300E8000053
:1091D00020202020205472696D203420202020205F
:1091E000006891B6910400E8000020202020416929
:1091F0006C65726F6E20202020200006920293077B
:10920000806E6515040020202020456C6576617411
:109210006F7220202020002292EA9107806E651B49
:1092200005002020202052756464657220202020D3
:109230002020003E92069207806E652106002020C5
:1092400020205468726F74746C6520202020005AAE
:109250009222920780A0642707002020202020204F
:10926000434836202020202020200076923E92077E
:1092700080B4633B0000202020202020434837207A
:109280002020202020200092925A920780B4633F31
:109290000100202041696C65726F6E207472696DE7
:1092A000202000AE9276920780B4632B0800204500
:1092B0006C657661746F7220207472696D2000CACB
:1092C0009292920780B4632F090020205275646443
:1092D000657220207472696D202000E692AE9207BC
:1092E00080B463330A00205468726F74746C652014
:1092F000207472696D20000293CA920780B46337AC
:109300000B00457869742020202020202020202078
:10931000202000EA91E6920300D9000020202020BE
:1093200043656E74657220202020202000002020DC
:109330002052696768742F446F776E2020200000E8
:10934000202020204C6566742F557020202020207E
:109350000000204672616D696E67202020526174A2
:109360006520007293AE9305C8D4023E6F20003290
:109370000000204672616D655261746544656665E2
:109380006374008E9352930B88D502506F00205067
:109390004C4C20205265662020467265712000AE3C
:1093A0009372930C8E0102626FA869486900455858
:1093B000495420202020202020202020202000523E
:1093C000938E930300D9000001000F00D20000002B
:1093D0000300D20000001E00D2000080121B0166B4
:1093E0000379013C012E03AE0113012603950162AE
:1093F000017300860412018B040701C80405012AC9
:10940000042901320237023B022F0200000800014A
:1094100004091019243140516400132433404B5483
:109420005B60636400010203060C1522334964008B
:109430001B31424F585E61626364000A141E283279
:109440003C46505A640014283C5064503C28140098
:1094500000050A0F14192837465564000F1E2D3CCD
:109460004B50555A5F640A0A0000109001FF00A596
:10947000E7C009F30000DC059411010203040000B9
:10948000FF5801000102830405060708090A0B8C36
:109490008D0E0F00000000000000000028000000FA
:1094A00000000000000000000000000000000000BC
:1094B00000000000000000000000000000000000AC
:1094C00000000000000000004D4F44454C203031AA
:1094D0002020202020202020000001B80B00013C8B
:1094E000190000000001B80B00013C190000000049
:1094F00001B80B00013C1900000000FEA00F19018B
:10950000D0070001B80B0001B80B0001B80B000137
:10951000B80B000132FF320032003200CEFFCE0025
:10952000CE00CE0000000014140000000A0A000063
:10953000000A0A0000000A0A0000F4010A00000004
:109540000A0A0000000A0A0000000A0A0000000AD5
:109550000A0000000A0A0000000A0A0000000A0AC5
:10956000000000000000000A0000000000020000EF
:109570000000000000FF0001028304050607898B3C
:109580004B8C0D8E8F0100081000074B8C040020BF
:109590000000000000FF0D0020002000200020003F
:1095A00020000001040910192431405164001324E3
:1095B00033404B545B606364000000000000000017
:1095C0000000000000000000020103040506070877
:1095D000000000000000000000000000000000008B
:1095E000000000000000000000000000000000007B
:1095F000000000000000000000000000000000006B
:10960000000000000000000000000000000000005A
:10961000000000000000000000000000000000004A
:10962000000000000000000000000000000000003A
:10963000000000000000000000000000000000002A
:10964000000000000000000000000000000000001A
:10965000000000000000000000000000000000000A
:1096600000000000000000000000000000000000FA
:1096700000000000000000000000000000000000EA
:1096800000000000000000000000000000000000DA
:1096900000000000000000000000000000000000CA
:1096A00000000000000000000000000000000000BA
:1096B00000000000000000000000000000000000AA
:0896C0000000000000000000A2
:00000001FF
